:04701F00010002303A
:106A9000AF50055074D02FF582E4341DF583E5998D
:106AA000F022D3E5309400E52F94002290000FE00F
:036AB0006403225A
:030003000258D4CC
:0B58D400C0E0C083C082C0D075D008C7
:1058DF00852E82852D83E493FF201404C4540FFF7B
:1058EF00430FF08F80C284D28500C2870000D28719
:1058FF00007580FF7580FEC284C28500C2870000DC
:10590F00D287007580FF30140CC214052EE52E705F
:09591F0006052D8002D214D2A865
:09592800D0D0D082D083D0E0324F
:03000B000219696E
:10196900C0E0C0F0C083C082C0D075D008758CD8E3
:10197900758A92D28C1242FA1263D3E531D394005C
:1019890040171531E53164056009E531640F6003DD
:10199900021B7B126CD5021B7B753114E54ED39467
:1019A900004002154EE54FD394004002154FE53A29
:1019B900D394004002153AE54BD394004002154BED
:1019C900154CE54C123A5E1B6D001B42011B1A02B5
:1019D9001AF2031A6F041A56051A3D061A24071A31
:1019E9000B0819F20900001B78D3E52C9400E52BAC
:1019F90094005003021B7BE52C152C704D152B020E
:101A09001B7BD3E5379400E53694005003021B7B1A
:101A1900E537153770021536021B7BD3E54894006C
:101A2900E54794005003021B7BE5481548700215F1
:101A390047021B7BD3E54A9400E549940050030211
:101A49001B7BE54A154A70021549021B7BD3E52A1F
:101A59009400E52994005003021B7BE52A152A709E
:101A6900021529021B7B7884E6FF7003021B7BEFBA
:101A7900B40105900524801BEFB40210126AA2403C
:101A89002FE53015307002152F021B7BEFB4030CC4
:101A9900900526E0F52FA3E0F5308028EFB4041275
:101AA900126AA2400BE53015307002152F021B7B1C
:101AB9008012EF64057003021B7BEFB4060C752FCF
:101AC90002753058788406021B7BEF6407600302B5
:101AD9001B7B126AA2400BE53015307002152F02EC
:101AE9001B7B78847600021B7BD3E5399400E538AB
:101AF90094004008E539153970021538D3E53C944E
:101B090000E53B9400406BE53C153C7002153B80B9
:101B190061D3E5579400E55694004008E5571557F9
:101B290070021556D3E5559400E55494004043E5F9
:101B3900551555700215548039D3E5359400E534AF
:101B490094004008E535153570021534301523D356
:101B5900E5339400E53294004018E53315337012EB
:101B69001532800EE551D39400400415518000755B
:0D1B79004C0AD0D0D082D083D0F0D0E03222
:03001300023B6E3F
:0D3B6E00C0E0C0F0C083C082C0D075D01090
:103B7B00E545C394504003023C3E202403023C3EE7
:103B8B00300C03023C3EE5A0540FF5587D077F0136
:103B9B00124F405067202364E545700DE558B40C77
:103BAB0008201105D211023C3E20034A2011471276
:103BBB003C4950047F0180027F0F126FA290000FCF
:103BCB00E0FF64016012EFB40302800C90000FE081
:103BDB00B40209123C4950047F80801290000FE020
:103BEB00B4020E7D037F07124F4040057FA01200E9
:103BFB0016754202D20390053CE0F53A7D087F052D
:103C0B00124F40501A90002BE0B55807202304D2D6
:103C1B00268020053EE53EAE3D700E053D800A0533
:103C2B003EE53EAE3D7002053D14F5828E83E558B0
:033C3B00F005454C
:103C3E00D0D0D082D083D0F0D0E0327D037F071277
:033C4E004F4022C2
:030023000264ACC8
:1064AC00C0E0C083C082C0D075D018309819C29893
:1064BC00E599B40A08126A90755000800AE550C339
:1064CC0094905003126A90309902C299D0D0D08225
:0564DC00D083D0E03286
:03003B000246A0DA
:0D46A000C0E0C0F0C083C082C0D075D0184B
:1046AD00C2CEE546C39410400302474A20250302BB
:1046BD00474A300C0302474AAFA07804EF08800147
:1046CD0023D8FDF55953590F7D077F02124F4050E6
:1046DD0035202332E546700CE559B40C0720130440
:1046ED00D213805920041920131690000FE0B40244
:1046FD000F7F0A126FA27F80120016754202D2043C
:10470D0090053CE0F53A7D087F05124F40501A9018
:10471D00002BE0B55907202304D22880200540E561
:10472D0040AE3F700E053F800A0540E540AE3F703C
:0D473D0002053F14F5828E83E559F0054614
:0B474A00D0D0D082D083D0F0D0E0327D
:104C7900E4F55AF55B755C1E755DFF855B82855AA7
:104C890083E0F55E635EFFE55EF0E0655E6003125A
:104C99007023635EFF855B82855A83E55EF0E0657C
:104CA9005E6003127023055BE55B7002055AE55DE2
:104CB900155D7002155CD3E55D9400E55C940050C8
:104CC900BA75985A758921758845758DE7758780F4
:104CD900758CD8758AEF75C90275C808753D1E753A
:104CE9003E60753F1E7540B075B701D2A9D2E8D2B2
:0F4CF900AA75C64C75EEFF75FEFFD2AF1267DBD2
:014D08002288
:0270230080FEED
:106A6D00202F0F90053AE0F54EE54ED394004012DD
:106A7D0080F7302F0D90053AE0F54FE54FD3940098
:036A8D0050F9229B
:106A250030310AD215900024E04420800DC2157F34
:106A350008126FE3900024E054DFF0FD7F247E0010
:046A4500126476223F
:102ECA008F6AE56A640170292030047F01805620E8
:102EDA003003022FC5122FD64003022FC5122FDE50
:102EEA00500C122FC6301503022FC5022FBB022F1A
:102EFA007BE56A640270202030047F02802720303C
:102F0A0003022FC5122FE64003022FC5126AAC70C6
:102F1A0003022FC5022F95E56A64036003022FC5D9
:102F2A002030057F03026FE3303024122FD6501F62
:102F3A00122FE6501A126AAC6015122FDE500B7F60
:102F4A000B122FEE201574022FBB7F03022FC23003
:102F5A003023122FFC501E7D017F02124F40401574
:102F6A007D017F07124F405008122FC620154C8052
:102F7A00407F018043303017122FFC40127D017FC1
:102F8A0002124F405009126AAC60047F0280293055
:102F9A0030297D017F01124F405020126AAC701B0C
:102FAA007D017F07124F40500D7F09122FEE201529
:102FBA000AD231026A257F01126FF6227F09126F47
:102FCA00F6900536E0F532A3E0F533227D017F0164
:102FDA00124F40227D017F07124F40227D017F025E
:102FEA00124F4022126FF6900536E0F532A3E0F553
:0A2FFA0033227D017F01124F4022B7
:104D0900C2957FFF126FE3124C797F0712640A5034
:104D19000512003E8003126191D28C7F0812640A49
:104D290050051243BA80FEC22B12696B9000D1E084
:104D3900FF7C117D00125CC5125E3890000FE0B453
:104D49000105122831801090000FE0FF6402600411
:104D5900EFB40303123265123E15301E11E542709D
:104D69000DE52754A060077FA0126FA2C21E7D0720
:104D79007F05124F404002C200E552C3940A50BB5E
:104D89003015B8E533453270B2C231126A2580ABAD
:104B5000EF253EFFEE353DCF2401FDE43FFC22AFC3
:104B60005A7E00EF2403FDEE33FC22E53E255AF584
:104B700082E4353DF58322E540255AF582E4353F50
:104B8000F58322E56F256DF582E4356EF583E0FF50
:104B9000E56F256DF582E4356EF58322E55A240232
:104BA000FFE433FE22E56C2401FFE433FEC3E56D30
:104BB0009FEE6480F874809822EF2540FFEE353F29
:104BC00022C2017FF47E01126D47E56C25E0F56C91
:104BD000756D0122E55C2EF582E4355BF583E0FD21
:084BE00022753D1E753E6022A6
:106D4700EF1FAA0670011ED39400EA9400400BE4DB
:0A6D5700FDEDC394C850E90D80F76C
:016D6100220F
:10535A008F5BE55BB401197D017F06124F40500C4B
:10536A009000B1E0FF7C0D7D00125CC578840622B6
:10537A00E55BB402131253CC50439000B2E0FF7CB9
:10538A000D7D20125CC58035E55BB404161253CC42
:10539A00500C9000B4E0FF7C0D7D60125CC57884EF
:1053AA00760622E55BB403197D027F06124F405050
:1053BA000C9000B3E0FF7C0D7D40125CC5788476CA
:0A53CA0001227D027F06124F4022EF
:104F4000BF0107900020E0FE8048BF0207900021CB
:104F5000E0FE803EBF0307900022E0FE8034BF04E5
:104F600007900023E0FE802ABF0507900024E0FEA2
:104F70008020BF0607900025E0FE8016BF0707903F
:104F80000026E0FE800CBF0807900027E0FE8002AC
:104F9000E4FEBD0103EE1322BD0204EEA2E122BD38
:104FA0000304EEA2E222BD0404EEA2E322BD050446
:104FB000EEA2E422BD0604EEA2E522BD0704EEA2A5
:074FC000E622BD0802EE33FA
:014FC70022C7
:101D8700124BE1900100E0F55A124B6BE0123A5EFC
:101D97001DB6011DEB021E20031E55041E8A051EDB
:101DA700BF061EF4071F24081F500900001F7A12E0
:101DB7004B6BA3E0B40A15E55A124B9EE545B507F0
:101DC7000BE4B506077D017F01021F38124B5FE563
:101DD700456D7001EC6003021F7A124B50C2297FD8
:101DE70001021F4D124B6BA3E0B40A15E55A124BC3
:101DF7009EE545B5070BE4B506077D017F02021F87
:101E070038124B5FE5456D7001EC6003021F7A12D3
:101E17004B50C2297F02021F4D124B6BA3E0B40A3D
:101E270015E55A124B9EE545B5070BE4B506077D48
:101E3700017F03021F38124B5FE5456D7001EC60AF
:101E470003021F7A124B50C2297F03021F4D124B08
:101E57006BA3E0B40A15E55A124B9EE545B5070B8F
:101E6700E4B506077D017F04021F38124B5FE54585
:101E77006D7001EC6003021F7A124B50C2297F0478
:101E8700021F4D124B6BA3E0B40A15E55A124B9E85
:101E9700E545B5070BE4B506077D017F05021F3849
:101EA700124B5FE5456D7001EC6003021F7A124B20
:101EB70050C2297F05021F4D124B6BA3E0B40A15D0
:101EC700E55A124B9EE545B5070BE4B506077D01BC
:101ED7007F06021F38124B5FE5456D7001EC60030A
:101EE700021F7A124B50C2297F06021F4D124B6BFD
:101EF700A3E0B40A14E55A124B9EE545B5070AE478
:101F0700B506067D017F078028124B5FE5456D709A
:101F170001EC705F124B50C2297F078029124B6B6F
:101F2700A3E0B40A0F124B6BA3A3E070077D017FF8
:101F370008024EB5124B5FE5456D7001EC70341227
:101F47004B50C2297F08020FFB124B6BA3A3E07013
:101F570022124B6BA3E024F96008147016E4FF0209
:101F670060587FF47E01126D477D5E7F021267B174
:031F77001243BA58
:011F7A002244
:101B8600753F1E7540B0900108E0F55A124B77E09C
:101B9600123A5E1BB8011BF0021C28031C60041CD1
:101BA60098051CD0061D08071D3B081D700900007E
:101BB6001D86124B77A3E0B40A13124B9CE546B57B
:101BC600070BE4B506077D017F01021D53AF5A12CC
:101BD6004B61E5466D7001EC6003021D86124BB940
:101BE600124B57D2297F01021D6D124B77A3E0B429
:101BF6000A13124B9CE546B5070BE4B506077D01B3
:101C06007F02021D53AF5A124B61E5466D7001EC1F
:101C16006003021D86124BB9124B57D2297F02026E
:101C26001D6D124B77A3E0B40A13124B9CE546B523
:101C3600070BE4B506077D017F03021D53AF5A1259
:101C46004B61E5466D7001EC6003021D86124BB9CF
:101C5600124B57D2297F03021D6D124B77A3E0B4B6
:101C66000A13124B9CE546B5070BE4B506077D0142
:101C76007F04021D53AF5A124B61E5466D7001ECAD
:101C86006003021D86124BB9124B57D2297F0402FC
:101C96001D6D124B77A3E0B40A13124B9CE546B5B3
:101CA600070BE4B506077D017F05021D53AF5A12E7
:101CB6004B61E5466D7001EC6003021D86124BB95F
:101CC600124B57D2297F05021D6D124B77A3E0B444
:101CD6000A13124B9CE546B5070BE4B506077D01D2
:101CE6007F06021D53AF5A124B61E5466D7001EC3B
:101CF6006003021D86124BB9124B57D2297F06028A
:101D06001D6D124B77A3E0B40A12124B9CE546B543
:101D1600070AE4B506067D017F078031AF5A124BEC
:101D260061E5466D7001EC7057124BB9124B57D2F4
:101D3600297F078032124B77A3E0B40A13124B9C1B
:101D4600E546B5070BE4B506077D017F08024EB5EB
:101D5600AF5A124B61E5466D7001EC7023124BB918
:101D6600124B57D2297F08020FFB124B77A3A3E031
:101D7600700E124B77A3E024F870057F01126058AD
:011D8600223A
:04496A008C5B8D5C79
:10496E00055CE55C7002055B14F5828C83E0F970E2
:10497E0003024A11EF7005124BE18009BF01067563
:10498E003F1E7540B0302946EF7007E9654560025D
:10499E00C322BF0107E965466002C322E4FEEEC3EF
:1049AE00995029EF700F124BD4E53E2E124B6FE04B
:1049BE006D6002C322EF6401700F124BD4E5402EDE
:1049CE00124B7BE06D6002C3220E80D2D3222029CF
:1049DE0033E4FEEEC3995029EF700F124BD4E53E2F
:1049EE002E124B6FE06D6016C322EF6401700F1232
:1049FE004BD4E5402E124B7BE06D6002C3220E803D
:044A0E00D2D322C31A
:014A12002281
:060FFB008F5BAB05AA04A8
:101001007D027F07124F405011E55BB4050C8B82C6
:101011008A83E0640570030212687D017F07124F25
:10102100405011E55BB4050C8B828A83E064067045
:1010310003021268C22AEB24FFF582EA34FFF5832A
:10104100E0F55D8B828A83E0FFF55EA3E0F9F55F51
:10105100EF123A5E107101107802107F03108604BE
:10106100108D05109406109B0710A208000010A710
:10107100755C01D22A802F755C02D22A8028755CAA
:1010810004D22A8021755C08D22A801A755C10D29C
:101091002A8013755C20D22A800C755C40D22A808C
:1010A10005755C80D22AE924FE700302116924F8D7
:1010B100605C2409600302117BE55BB401059000CB
:1010C100208045E55BB40205900021803BE55BB4DF
:1010D10003059000228031E55BB404059000238074
:1010E10027E55BB40505900024801DE55BB406058A
:1010F1009000258013E55BB407059000268009E583
:101101005B64087077900027E0455CF0806EE55BDA
:10111100B401059000208045E55BB40205900021F3
:10112100803BE55BB403059000228031E55BB404AC
:10113100059000238027E55BB40505900024801D00
:10114100E55BB406059000258013E55BB4070590C7
:1011510000268009E55B64087022900027E0FFE526
:101161005CF4FEEF5EF08014E55BB4050D8B828AC2
:1011710083E0FFD22F122992C22AC22A202A030217
:101181001268E55BB40109900020E0FD7F208060DA
:10119100E55BB40209900021E0FD7F218052E55B0F
:1011A100B40309900022E0FD7F228044E55BB40492
:1011B10009900023E0FD7F238036E55BB4050990AB
:1011C1000024E0FD7F248028E55BB406099000251A
:1011D100E0FD7F25801AE55BB40709900026E0FD5C
:1011E1007F26800CE55BB4080C900027E0FD7F278B
:1011F1007E00126476126E41D2AF2029047F0180F5
:10120100027F02126FF6A229922F126A6DAD5DE480
:10121100FF1267B1AD5EE4FF1267B1E55FB401048F
:101221007D388007E55FB40A077D367F061267B116
:10123100E55BB4050312660E7D077F05124F405032
:101241000A200007C2307F03122ECA7D017F0112DE
:101251004F404005C230122ECA7D017F02124F401D
:071261004005C230122ECA45
:011268002263
:024EB5008F5B11
:104EB700ED24FF922F126A6DE55B123A5E4EE00118
:104EC7004EE5024EEA034EEF044EF4054EF9064E48
:104ED700FE074F030800004F099000208021900033
:104EE70021801C90002280179000238012900024BC
:104EF700800D90002580089000268003900027E011
:104F0700F55CE55C6024755E01E4F55DE55C30E029
:104F170007AD5EE4FF1267B1E55CC313F55C055EA0
:104F2700055DE55DC3940840E3227D187F021267A3
:084F3700B17D537F021267B146
:014F3F00224F
:10640A00C2AFD284C285BF070BC28600E580A2E272
:10641A00922A8019BF080BC28600E580A2E3922A5D
:10642A00800BBF0508C28600E58013922AD286D265
:05643A0085D2AFA22A8B
:01643F00223A
:10475500C229D22DE4FF125AF27D2E7F031267B1D2
:104765007D607F021267B17F03126FE33024FD2065
:1047750024FDE5456407703B7E017F50124BE18FB8
:10478500828E837407F07D01E53E2D124B6FE58225
:1047950024FFF582E58334FFF583E0F9EF2DF582FB
:1047A500E43EF583E9F00DBD08DED2297F647E0085
:1047B500126D477F0812640A5043302995D22DE4C3
:1047C500FF125AF27D607F021267B17D327F0612B9
:1047D50067B17D1E7F051267B1C22DE4FF125AF243
:1047E5007C017D507B087F507E011256EE7F0812BA
:1047F500640A50097F327E00126D4780F07F647E27
:0448050000126D47E9
:01480900228C
:0255A7008F5A19
:1055A900900138E0F55BE55A7020E55B124B9EE50A
:1055B900456F7001EE70547460255BF582E4341E0A
:1055C900AF82F55D8F5E7F408024E55A6401703BB0
:1055D900E55B124B9EE5466F7001EE702E74B025A7
:1055E9005BF582E4341EAF82F55D8F5E7F10120099
:1055F90016855E82855D83E0FFA3E0FD126E8F8FC5
:0B5609005CE4FD12504F7F50126FA2B6
:015614002273
:02504F008D6B67
:1050510075F020EF900280123A52AF8285836E8FF5
:105061006FE0F56CD394004063E56C9410505DE5FE
:105071006B7014124BC3124BA55051124B8312503B
:10508100CE056D056D80EFE56B6401701C124BC19F
:10509100124BA55037124B831250CE3024057F504E
:1050A100026FA2056D056D80E7E56B6402701D124C
:1050B1004BC1124BA55015124B83A3E0FD12663E66
:0C50C100302403024173056D056D80E68C
:0850CD0022A3E0FD12663E2261
:100D2E00855C82855B83A3A3E0FF855C82855B8304
:100D3E00A3222430F58274003EF583EDF0AF62EF0E
:100D4E003395E0FEE55F2FF582E55E3EF58322E505
:100D5E00822406F582E43583F583E0FF126E6AADD8
:100D6E0007AF63EF3395E0FEEF22A3A3E0FFE55C50
:100D7E002404F582E4355BF583E022E55F2405F576
:100D8E0082E4355EF583E022E55F2405F582E435E5
:100D9E005EF583E0FFE55F2406F582E4355EF583BC
:100DAE00E0228E69F56AAF68EF3395E0FEE5662FB7
:100DBE00F582E5653EF583222455F582E4340AF585
:100DCE0083EFF0E56275F007A422AF60EF3395E094
:100DDE00FEE56175F008900158123A52E5822FF542
:100DEE0082E5833EF58322E5662405F582E43565CA
:100DFE00F583E022E55E75F007A42454F582E43411
:100E0E000AF58322A3A3A3E0FF8D828C83E58224BF
:100E1E0004F582E43583F583E022E55E75F007A4E0
:100E2E002451F582E4340AF5832224E0F582740A13
:100E3E003EF583E5822DF582E5833CF58322E55E62
:100E4E0075F007A42453F582E4340AF58322E55F96
:100E5E002405F582E4355EF583E0FFE55F2406F5B3
:100E6E0082E4355EF583E022E55E75F007A4245238
:100E7E00F582E4340AF58322749F2562F582E43408
:100E8E0000F58322746F2562F582E43400F5832227
:100E9E002450F582E4340AF58322ECFF3395E0FE0C
:100EAE00EF25E0FFEE33FE75F02022E5602405F518
:100EBE0082E4355FF58322D3EF6480948022AB0702
:100ECE00AA068B828A83A3A3A3E0FFEB2404F582F8
:100EDE00E43AF583E0FD228F828E83A3A3A3E02262
:100EEE00855F82855E83A3A322AB5DAD5AAF5CAEF8
:100EFE005B22FFE562FD3395E0FCE55F2DF582E5B3
:100F0E005E3CF5832233CE33CE92E022A2E0CE13A6
:100F1E00CE132275F00AA42DFDE5F03CFCE5662209
:100F2E00E5602405F582E4355FF583E022E5627520
:100F3E00F008900158023A52E55E75F007A4245568
:100F4E00F582E4340AF583E022AB5AAD5DAF5CAEB8
:100F5E005B22EF7C002563FDEC35628D82F58322EA
:100F6E00A3A3E0FFAD5A22540FF5657808AF03AE88
:100F7E0002EF08220564E564AE632275F020123A92
:100F8E0052E0FEA3E0FF22E0FAA3E0FB780CFFAEF6
:100F9E00020822E0FCA3E0FD7804FFAE040822E57F
:100FAE00632561F582E43562F58322E5662DF582CF
:100FBE00E5653CF58322E5662FF582E5653EF58312
:100FCE00222431F5827400222480F58274023EAF11
:100FDE0082222560F560E4355FF55F2285608285AB
:0D0FEE005F83228F828E83A3A3E0640A221A
:02055B008F5AB5
:10055D00C22AE4F542D223D22D125AF27D4B7F02EC
:10056D001267B17D02E4FF1267B17D32E4FF1267BD
:10057D00B17D607F021267B17D027F07124F40503F
:10058D00057F04126FE3900528E0F536A3E0F537FB
:10059D007F03126FE3E55A7006A22492298009E5C4
:1005AD005AB40104A2259229E53745367005D22AA1
:1005BD00020A223029DFE55A7006A2249229800909
:1005CD00E55AB40104A22592292029EAE55A700BB7
:1005DD00755B1E755C6085455D800EE55AB401093D
:1005ED00755B1E755CB085465DE55DD3940050036B
:1005FD00020A1C855C82855B83E0640B6003020A42
:10060D0017A3E0FFB40A0AE55DB40205D22A020A77
:10061D001CEF6401701E120D38A3E0640A7015E51D
:10062D005D6405700F120D38120D78120A4D1231DE
:10063D0038020A1C120D38E0B40111120D38A3E076
:10064D00B40109120EF7121725020A1C120D38E01B
:10065D006401701E120D38A3E064027015E55D642F
:10066D0005700F120D38120D78120A4D12627F02AD
:10067D000A1C120D38E06401701D120D38A3E064E0
:10068D00037014E55DB4050F120D38120D78FDAB36
:10069D005A123A84020A1C120D38E0B4011D120DD3
:1006AD0038A3E0B40415E55DD39405400EAB5AAD07
:1006BD005CAC5BAF5D123004020A1C120D38E064B5
:1006CD0001701D120D38A3E064057014E55DB405CD
:1006DD000F120D38120D78FDAB5A125BE4020A1C95
:1006ED00120D38E06401701D120D38A3E064067020
:1006FD0014E55DB4050F120D38120D78FDAB5A12CD
:10070D004E28020A1C120D38E0B4011D120D38A33B
:10071D00E0B40715E55DD39405400EAB5AAD5CAC66
:10072D005BAF5D12480A020A1C120D38E0640170BD
:10073D001D120D38A3E064087014E55DB4050F12A9
:10074D000D38120D78FDAB5A1262B9020A1C120D4A
:10075D0038E0B40215120D38A3E0B40A0DE55DB40E
:10076D000308AF5A126440020A1C120D38E0B4029D
:10077D0016120D38A3E0B4010EE55DB40E09120E8C
:10078D00F9122D8E020A1C120D38E0B40216120D4C
:10079D0038A3E0B4020EE55DB40709120EF9125448
:1007AD004D020A1C120D38E0B40215120D38A3E0EB
:1007BD00B4090DE55DB40308AF5A125682020A1C46
:1007CD00120D38E064027019120D38A3E0B409114E
:1007DD00E55DB4040C120D38120F6E126857020A43
:1007ED001C120D38E064037021120D38A3E0640A69
:1007FD007018E55D64057012120D38120D78FD123A
:10080D006E8FAD5A1248BF020A1C120D38E06403F8
:10081D007029120D38A3E064017020E55DD39405B5
:10082D004019120D38120D78FD126E8F855A62AB7C
:10083D005DAD5CAC5B123EF6020A1C120D38E06435
:10084D00037021120D38A3E064027018E55D640594
:10085D007012120D38120D78FD126E8FAD5A126096
:10086D00D8020A1C120D38E0B40315120D38A3E09E
:10087D00B4030DE55DB40308AF5A126154020A1CAE
:10088D00120D38E0B40318120D38A3E0B40410E5CE
:10089D005DD394034009120F57124AB7020A1C1276
:1008AD000D38E0B40315120D38A3E0B4050DE55D68
:1008BD00B40308AF5A126E7D020A1C120D38E0B453
:1008CD000316120D38A3E0B4060EE55DB40509124A
:1008DD000EF9126991020A1C120D38E064037019A9
:1008ED00120D38A3E0B40711E55DB4040C120D38F8
:1008FD00120F6E126C9B020A1C120D38E0B4031617
:10090D00120D38A3E0B4080EE55DB40409120EF91A
:10091D001269B6020A1C120D38E064057014E55D0B
:10092D00B4040F120D2EA3A3E0FDAB5A121F7B02D0
:10093D000A1C120D38E0B40516120D7CB40B10E52F
:10094D005DD394054009120F57123391020A1C1200
:10095D000D38E064067014E55DB4040F120D2EA37E
:10096D00A3E0FDAB5A12216D020A1C120D38E0B442
:10097D000616120D7CB40B10E55DD39405400912DB
:10098D000F571226A8020A1C120D38E06409701ABE
:10099D00120D38A3E0B40A12E55DB4040D120D3842
:1009AD00A3A3E0FF125E81020A1C120D38E0640958
:1009BD007018120D38A3E0B40110E55DB4040B12EC
:1009CD000D38120F6E12639C8045120D38E0B4097C
:1009DD0017120D38A3E0B4020FE55DD3940440085F
:1009ED00120EF71214D78027120D38E06409701A11
:1009FD00120D38A3E0B40310E55DB4040B120D38ED
:100A0D00120F6E125DEF80078000AF5A126CB82086
:100A1D002A030205A2C21ED22DAF5A125AF27D60D0
:100A2D007F021267B17D327F031267B17F03126FB0
:0F0A3D00E3125EC97FFF126FA2E47884F6C22332
:080A4C0022FD126E8FAD5A224B
:081725008E5E8F5F8D608B6109
:10172D00120EE5FFE55F2404120D8DFD1265498F44
:10173D006274E22562F562C394005003021926E536
:10174D006294144003021926E5616406701D120DA2
:10175D0089B4010C120DD1120E9E7401F0021922E2
:10176D00120DD1120E9EE4F0021922E561640E6095
:10177D0003021844E55F240C120D8DFFB40A14E525
:10178D005F240D120D8DB40A0A120DD1120E2EE426
:10179D00F08013E55F240D120D8DFD126D0F120DEE
:1017AD00D1120E2EEFF0E55F240A120D8DFFB40A53
:1017BD0014E55F240B120D8DB40A0A120DD1120E11
:1017CD007CE4F08013E55F240B120D8DFD126D0F7F
:1017DD00120DD1120E7CEFF0E55F2409120D8DFF75
:1017ED00640A6006EFD39409400A120DD1120E520D
:1017FD00E4F08010E55F2409120D8DFF120DD1125A
:10180D000E52EFF0120D89FFB40B15E55F24061291
:10181D000D8DB40B0B120DD1120E0874FFF0800854
:10182D00121952120E08EFF012192E120DC6120EC9
:10183D009E7401F0021922E561640A706E120DD1D9
:10184D00120E2EE4120DD0120E7CE4F0E55F240989
:10185D00120D8DFF640A6006EFD39409400A120D34
:10186D00D1120E52E4F08010E55F2409120D8DFFA8
:10187D00120DD1120E52EFF0120D89FFB40B15E5BA
:10188D005F2406120D8DB40B0B120DD1120E0874C0
:10189D00FFF08008121952120E08EFF012192E12D5
:1018AD000DC6120E9E7401F0021922E561640970D5
:1018BD0068120DD1120E2EE4120DD0120E7CE41210
:1018CD000DD0120E52E4F0120D89FFB40B15E55F29
:1018DD002406120D8DB40B0B120DD1120E0874FFD0
:1018ED00F08013E55F2406120D8DFD126D0F120DA4
:1018FD00D1120E08EFF0E55F2407120D8DFFE55FA5
:10190D002408120D8DFD126D0F120DD1120DC61280
:10191D000E9E7401F0D22C8002C22CAF60126F7833
:10192D0022E55F2407F582E4355EF583E0FFE55F90
:10193D002408F582E4355EF583E0FD126D0FE56256
:10194D0075F007A422E55F2406F582E4355EF58384
:0C195D00E0FD126D0FE56275F007A4229A
:103138008F5E8D5FE55ED3941D5003023244E55ED9
:1031480094324003023244D22DAF5F125AF27D46C8
:103158007F071267B1AF5E1235B874E2255EF55E7F
:10316800120E2AE07021120E76E0701B120E4CE04F
:103178007015120E02E0700F120F46700A12325DBF
:103188007D537F0202323A12324CE55E75F007A495
:10319800120E9EE070047D3680027D387F0612672D
:1031A800B112324C120E28E0FFD394014034EF9450
:1031B80013502F7D097F061267B1120E2812325460
:1031C8007FF47E01126D477D0E7F031267B17D3556
:1031D8007F061267B17D097F061267B1120E76125B
:1031E80032547FF47E01126D47120E4CE0FF6005E9
:1031F800125B95800A12325D7D0F7F031267B17DE5
:10320800277F021267B1120E02E0FFF46008126D08
:10321800CC1235B880077D187F021267B17D377FE1
:10322800041267B1120F46FF126DCC1235B87D0536
:103238007F061267B1C22DAF5F025AF2C22CAF5F90
:10324800126F78227FF47E01126D4722E0FF126D23
:0D325800CC1235B8227D187F021267B1221A
:02627F008D5E32
:10628100EFD3941D402AEF9432502574E22FFFE49E
:10629100FEEEFD3395E0FCEF75F007A42450F58286
:1062A100E4340A120E3FE4F00EBE07E5D22C800260
:0762B100C22CAF5E126F78F2
:0162B80022C3
:062D8E008E5E8F5F8D6078
:102D9400D22B120EE5FFE55F2404120DA7122EB507
:102DA400C39418501C855F82855E83A3A3A3E0FFB0
:102DB400E55F2404120DA7FD126E577882A60780E2
:102DC40006E47882F6C22B120D96122EB5C3943CFB
:102DD400500D120D96FD126E577883A6078006E4F7
:102DE4007883F6C22BE55F2407120DA7FF126F0A42
:102DF4008F61E561D394004017E56194085011E5B3
:102E04005F2407120DA7FF126F0A787FA6078006BA
:102E1400787F7601C22BE55F2408120DA7FFE55FDA
:102E24002409120DA7122EBE401FE56194205019EB
:102E3400E55F2408120DA7FFE55F2409120DA7FD25
:102E4400126E577887A607800678877601C22BE52D
:102E54005F240A120DA7FFE55F240B120DA7122EA3
:102E6400BE401FE561940D5019E55F240A120DA7B9
:102E7400FFE55F240B120DA7FD126E577880A6079D
:102E8400800678807601C22BE55F240C120DA7FF23
:102E9400E55F240D120DA7FD126E577881A6073049
:102EA4002B071259E9D22C8002C22CAF60126F7822
:102EB40022FD1265498F61E56122FD1265498F612A
:062EC400E561D394002239
:06544D008E5E8F5F8D6092
:10545300D22B120EE5FFE55F2404120E6D1254B831
:105463009418501C855F82855E83A3A3A3E0FFE5A8
:105473005F2404120E6DFD126E577882A607800614
:10548300E47882F6C22B120E5C1254B8943C500D91
:10549300120E5CFD126E577883A6078006E47883AC
:1054A300F6C22B302B071259E9D22C8002C22CAF43
:0454B30060126F789C
:0B54B70022FD1265498F61E561C322F0
:106F0A00120EC54008EF6480948A5001227F002245
:106E5700AE05126F0AEFC454F0FDAF06126F0AEFCA
:036E67004DFF22BA
:106440008F5ED22D125AF27D1E7F081267B17D2613
:106450007F081267B17D527F041267B1C22B1269A7
:106460006B125D5B787FE6FF125B95125A9CC22D22
:06647000AF5E125AF22299
:106857008D5EEFD3940A4006EFD3940F4003EF7099
:106867000E90002BEFF0D22CAF5E126F78D322C2BE
:086877002CAF5E126F78C32202
:025682008F5E39
:10568400D22D125AF27D207F051267B17D2E7F0341
:105694001267B17D527F041267B190002BE0F55F71
:1056A400E55FB40B067D5F7F078034E55FB40C06CD
:1056B4007D5E7F068029E55FB40D067D0A7F02804A
:1056C4001EE55FB40E067D327F028013E55FB40FE2
:1056D400067D467F028008E55F70077D0A7F03121E
:0956E40067B1C22DAF5E125AF24B
:0156ED00229A
:106C9B008D5E120EC5400EEF648094865007126411
:0D6CAB00E1D22C8002C22CAF5E126F782265
:026991008D5E19
:10699300120ECC126549120EC54010EF648094A10B
:1069A3005009900029EFF0D22C8002C22CAF5E1266
:0269B3006F78FB
:0169B50022BF
:0269B6008D5EF4
:1069B800120ECC126549120EC54010EF648094A1E6
:1069C8005009900028EFF0D22C8002C22CAF5E1242
:0269D8006F78D6
:0169DA00229A
:106E6A00D3EF648094814008EF6480948A500122B1
:036E7A007F002274
:106F1A00120EC54008EF648094A15001227F00221E
:0814D7008E5E8F5F8D608B615A
:1014DF00120EE514F56374FC2561F5616403600F6A
:1014EF00E56164076009E561640B60030216C2C31E
:1014FF00E5636480948050030216C2E563648094B0
:10150F008840030216C2E4F562120D6F7803C333ED
:10151F00CE33CED8F92430F58274003EF583AF6216
:10152F00EF3395E0FE120DEAE4F00562E562B408D0
:10153F00D8756204E56164037029120D4B12170808
:10154F00120D6D7803C333CE33CED8F9120D40A3ED
:10155F00A3120D687803C333CE33CED8F9120FCF51
:10156F000216B9E56164077069120D4B1217081264
:10157F000D6D7803C333CE33CED8F9120D40A3A32C
:10158F00120D687803C333CE33CED8F9120FCF12B2
:10159F000D46A3A3A3120D687803C333CE33CED861
:1015AF00F92432F5827400120D461216CAC333CED7
:1015BF0033CED8F92433F5827400120D46120D5D27
:1015CF007803C333CE33CED8F92434F582740002B6
:1015DF0016B9E561640B60030216C2120D4BE012DF
:1015EF000F00A3E0FD126549126F1A120D6D7803FB
:1015FF00C333CE33CED8F9120D40A3A3120D6878A2
:10160F0003C333CE33CED8F9120FCF120D46A3A397
:10161F00A3120D687803C333CE33CED8F92432F535
:10162F00827400120D461216CAC333CE33CED8F9C8
:10163F002433F5827400120D46120D5D7803C33307
:10164F00CE33CED8F92434F5827400120D46E582DC
:10165F002407120D617803C333CE33CED8F9243566
:10166F00F5827400120D46E5822408120E1F120F28
:10167F0000E5822409120E1FFD126549126F1A121E
:10168F000D6D7803C333CE33CED8F92436F582747B
:10169F0000120D46E582240A120D617803C333CE82
:1016AF0033CED8F92437F58274003EF583EDF0D2AE
:0A16BF002C8002C22CAF60126F787D
:1016C90022E5822404F582E43583F583E0FFE562AF
:1016D900FD3395E0FCE55F2DF582E55E3CF583E59C
:1016E900822405F582E43583F583E0FD126549120C
:1016F9006F1AAD07AF63EF3395E0FEEF780322E091
:10170900FFE562FD3395E0FCE55F2DF582E55E3C82
:0C171900F583A3E0FD126549126F1A224F
:045DEF008D5EAC0712
:105DF300D3EC648094804035EC64809489502EE425
:105E0300FDECFF3395E0FEEF7803C333CE33CED8FA
:105E1300F92428F58274003EF583EDFF3395E0FE07
:105E2300120DEAE4F00DBD08D8D22C8002C22CAFCB
:045E33005E126F7814
:015E37002248
:10639C008D5E120EC5402FEF648094895028EF1447
:1063AC00FFE55E24FF922B1250D5D22DAF5E125A10
:1063BC00F27542017F327E00126D47E54270FCC2DD
:0763CC002DAF5E125AF22210
:08480A008F5E8C5F8D608B61F5
:10481200856082855F83120E12FD1265498F62E503
:1048220062D3940050030248B7E562943340030216
:1048320048B7E55E64067036D22DAF61125AF27D3A
:10484200527F051267B1AF621235B8120F2EB40152
:104852000A120E867401F07D388007120E86E4F08B
:104862007D367F061267B1C22DAF61025AF2E56052
:104872002406120F32640B703C120F2EB401081280
:104882000E867401F08005120E86E4F074F9255E3E
:10489200F55E75F004123998AFF0EF7014E56024FC
:1048A20006FBE4355FFAAD62E4FF1234B8D22C8025
:0C48B20006C22C8002C22CAF61126F788D
:0148BE0022D7
:083004008F5E8C5F8D608B6113
:10300C00856082855F83120E12FD1265498F62E521
:10301C0062D394005003023130E5629429400302DC
:10302C003130E55E64067037D22DAF61125AF27DF5
:10303C00527F051267B1AF621235B8120EB9E0B407
:10304C00010A120E927401F07D388007120E92E480
:10305C00F07D367F061267B1C22DAF61025AF2E5E0
:10306C00602406120EBDE0640B6003023130120EB8
:10307C00B9E0B40108120E927401F08005120E92A0
:10308C00E4F0E4FFFEE5602407120EBDE5822E128B
:10309C000E1FB40B04AF0680040EBE08E8EF7003DD
:1030AC00023130C39408507C120F3BEFF07E01EFDD
:1030BC002401FDE433FCEEC39DEC6480F87480982D
:1030CC005020E5602406120EBDE5822E120E1FFD67
:1030DC00120F3BE5822EF582E43583F583EDF00E7D
:1030EC0080CDE5602408120EBDE5822F120E1F6400
:1030FC000B602DEF2408FEC3E55E9EF55E75F004B3
:10310C00123998AEF0EE701CE5602407FDE4355FD3
:10311C00FC7E00ED2FFBEE3CFAAD627F011234B861
:0B312C00D22C8002C22CAF61126F7821
:013137002275
:0834B8008F638D648A658B6649
:1034C000756801E4F567120DB4E0FF6409703E12FF
:1034D00035A98003120F13D8FB120DB012359B785B
:1034E00008EF088003120F13D8FB120DB0A3A3E05E
:1034F000FFE568FD3395E0FCE5662DF582E5653C6A
:10350000F583A3A3A3E0FD126E8F023554120DB410
:10351000E0FF1235A98003120F13D8FB120DB01271
:10352000359B7804EF088003120F13D8FB120DB0FF
:10353000A3A3E0FF126FD9EF426AAE69AF6A7804C5
:10354000EF088003120F13D8FB120DB0A3A3A3E062
:10355000FF126FD9EF426AE563700FAF67120D710A
:10356000120EAFE564900AC08012E563B40117AF94
:1035700067120D71120EAFE564900530120DE7E58C
:1035800069F0A3E56AF074042568F5680567C3E58A
:0A359000676480949050030234C673
:10359A0022A3E0FF126FD9EF426AAE69AF6A221224
:0E35AA006FD97569008F6AAE697804EF082248
:0A6FD900EFD3940940037F00222249
:023A84008B5E57
:103A86001265498F61E561D394005003023B66E5F8
:103A96006194334003023B66D22DAF5E125AF27D2B
:103AA600527F051267B1AF611235B8746F25611286
:103AB6000E96E060047D3880027D367F061267B17F
:103AC6007F2C7E01126D47E561120F3DE0F55F70B8
:103AD600077D1B7F061267B17D577F021267B1E52E
:103AE6005F603B756001AF5F120D712401FFE43E1C
:103AF600FEAD60ED3395E0FCC3ED9FEE6480F8EC1F
:103B06006480985019120DD8E0B40A04E4FD8006CA
:103B1600120DD8E0FDE4FF1267B1056080C87F2C66
:103B26007E01126D47E561900530120F8990000005
:103B3600EEF0A3EFF04E70077D1B7F061267B17D96
:103B46000C7F031267B1900000E07002A3E06009E9
:103B5600E56114FD7F01122AF0C22DAF5E025AF212
:073B6600C22CAF5E126F7864
:013B6D002235
:024E28008B5E9F
:104E2A001265498F5FE55FD394004077E55F94335D
:104E3A005071D22DAF5E125AF27D527F051267B1C0
:104E4A00AF5F1235B8749F255F120E8AE060047D49
:104E5A003880027D367F061267B17F2C7E01126D83
:104E6A00477F2C7E01126D47E55F900AC0120F89B9
:104E7A00900000EEF0A3EFF04E70077D1B7F061244
:104E8A0067B17D0C7F031267B1900000E07002A346
:104E9A00E06009E55F14FDE4FF122AF0C22DAF5E5F
:0A4EAA00025AF2C22CAF5E126F78BC
:014EB40022DB
:0262B9008B5EFA
:1062BB00126549AD07EDD394004025ED9433502082
:1062CB00E4FC120EA8ED900AC0120DE7E4F0A3F067
:1062DB000CBC10EE749F2D120E8AE4F0D22C8002AF
:0762EB00C22CAF5E126F78B8
:0162F2002289
:025BE4008B5ED6
:105BE600126549AD07EDD394004036ED943350313C
:105BF600E4FC120EA8ED900530120DE7E4F0A3F0D8
:105C06000CBC10EE746F2D120E96E4F0FCECFF3314
:105C160095E0FEED120DE1E4F00CBC08F0D22C800C
:085C260002C22CAF5E126F7880
:015C2E002253
:042AF0008F628D6301
:102AF400E4F564E5627052AF64120D7125E0FDEEF9
:102B040033FCAF63120D717805C333CE33CED8F9DD
:102B1400120E38120F958003120F1AD8FB120F757C
:102B24008003120F1AD8FB540FF566AF63120D71B0
:102B34007805C333CE33CED8F9120E38120FA180E4
:102B440003120F1AD8FB022BAEE56264017064AF66
:102B540064120D7125E0FDEE33FCAF63120D717844
:102B640005C333CE33CED8F92450F5827405120E42
:102B74003E120F958003120F1AD8FB120F758003B3
:102B8400120F1AD8FB540FF566AF63120D71780556
:102B9400C333CE33CED8F92450F5827405120E3ED9
:102BA400120FA18003120F1AD8FB540FF567ED54CE
:102BB4000FF568E565700CE5667008E5677004E577
:102BC40068607CAD65E4FF1267B1AD66E4FF12672F
:102BD400B1E56564097045856769AF69FE7804EFFE
:102BE400088003120F13D8FBF569E5684269E569AB
:102BF400B4990B7D09E4FF1267B17D098027E5696B
:102C040075F00A84F56AFDE4FF1267B1E56A75F0B0
:102C14000AA4FFC3E5699FF56AFD8009AD67E4FF77
:102C24001267B1AD68E4FF1267B17FF47E01126DE3
:0F2C3400470564C3E564648094A05003022AF747
:012C4300226E
:10654900EFD394004015EF940B5010EFC3940A5009
:1065590008EF75F00AA4FE8002E4FEEDD394004032
:106569000EED940B5009EDC3940A5003ED2EFEAFC6
:01657900061B
:01657A0022FE
:064AB7008E5E8F5F8B6034
:104ABD00756105756240D3ED64809484407CED642E
:104ACD008094A55075ED24FDF563D39404406BE5FA
:104ADD006320E06613F5640562E562AE6170020560
:104AED006114F5828E83E564F07403255FF55FE450
:104AFD00355EF55EE4F563E563C395645033855F1C
:104B0D0082855E83E0FFA3E0FD126E8F0562E56294
:104B1D00AC617002056114F5828C83EFF0055FE5E1
:104B2D005F7002055E055FE55F7002055E056380DF
:104B3D00C6D22CAF60126F78D322C22CAF60126F29
:024B4D0078C32B
:014B4F002243
:043EF6008C5F8D60F0
:103EFA00120EC55003023FCEEF6480949540030230
:103F0A003FCEEB648094875003023FCEEB648094EB
:103F1A00E44003023FCE120D717805C333CE33CE8F
:103F2A00D8F9120FD6F5638F64EB24FBF565D394A9
:103F3A00025003023FCEE56575F00384E5F06003A5
:103F4A00023FCEE56575F00384F567C3941050749B
:103F5A00120F827002056314F5828E83E567F0748E
:103F6A0005120FE0E4F565E565C395675052120F37
:103F7A00EAE0F566B40A10120F827002056314F5BE
:103F8A00828E83E4F0800F120F827002056314F5AB
:103F9A00828E83E566F0120FEAA3E0FF120FEAA30E
:103FAA00A3E0FD126E8F8F66120F827002056314F2
:103FBA00F5828E83E566F07403120FE0056580A72B
:0B3FCA00D22C8002C22CAF62126F7874
:013FD50022C9
:0826A8008E5E8F5F8D608B6177
:1026B000C22B120FF160030227451228205003029B
:1026C0002740E5649408E56394075074C3E56064AB
:1026D00080948A506B120EEEA3E0F562B40106906E
:1026E0000520022795E562B402069005220227958F
:1026F000E562B40306900524022795E562B404065A
:10270000900526022795E562B40506900528022764
:1027100095E562B4060690052A022795E562B4079E
:102720000690052C022795E562B4080590052E80D9
:1027300064E562B40905900530805AD22B02281155
:10274000D22B022811120EEEE064017052AD60AF80
:102750005FAE5E1228205003022811E5649408E55C
:102760006394074003022811C3E5606480948A40A3
:1027700003022811120EEEA3E0F562B40A059005DB
:10278000328012E562B401059005348008E562B438
:102790000209900536E563F0A3806FD22B80721298
:1027A0000EEEE06402706AAD60AF5FAE5E125C2F49
:1027B0007563008F64C3E5649463E56394005051CE
:1027C000C3E560648094885048120EEEA3E0F56281
:1027D000B40107900538EFF08037E562B402059048
:1027E00005398026E562B4030590053A801CE56250
:1027F000B4040590053B8012E562B4050590053CE4
:102800008008E562B4060890053DE564F08002D2D8
:0F2810002B302B04C22C8002D22CAF61126F78B8
:10281F0022124A138E638F64D3E564943BE563946D
:02282F00002285
:064A13008E658F66A90507
:104A19007D057C00120FB9E0C3940A4005120FB955
:104A2900E4F00DBD00010CED640A4C70E7B906070E
:104A3900120DF5FF7E0022E964077010120DF5755D
:104A4900F00AA4ACF0FDE5662406801BE964087051
:104A590021120DF575F064A4ACF0FDE5662406128B
:104A69000DF9120F212407120DF92DFDE43CAF05B4
:104A7900FE22E964097033120DF5FF7E007C037D87
:104A8900E81239BAAC06AD07E5662406120DF975C8
:104A9900F064120F242407120DF9120F21240812B1
:0D4AA9000DF92DFDE43CFEAF0522E4FEFFFB
:014AB60022DD
:065C2F008E658F66A905D9
:105C35007F057E00120FC4E0C3940A4005120FC40D
:105C4500E4F00FBF00010EEF64084E70E7E964074A
:105C55007020E5662405F582E43565F583E075F089
:105C65000AA4FFE5662406F582E43565F583E02F91
:045C7500FF227F008B
:015C79002208
:083391008E5E8F5F8D608B6181
:10339900C22BD3E56064809484500302343FE56016
:1033A9006480948D400302343F120FF160030234AC
:1033B9003F120EE5123A5E33DF0133EA0233F503B9
:1033C90033FF04340905341306341D073427083440
:1033D90031090000343B756201756300D22B023458
:1033E90076756201756308D22B02347675620175B0
:1033F9006310D22B8077756201756318D22B806DAB
:10340900756201756320D22B80637562017563282B
:10341900D22B8059756201756330D22B804F75624A
:1034290001756338D22B8045756201756340D22BD3
:10343900803BC22B8037D3E56064809484402EE5BD
:10344900606480948D5026855F82855E83A3A3E0A6
:10345900B4011A855F82855E83A3A3A3E024F67075
:103469000A756201756358D22B8002C22B302B3743
:10347900E4FF120F60E4F00FBF08F7E56024FB8555
:103489006382856283F07F01E55F2404F582E43578
:103499005EF583E5822F120E1FFE120F60EEF00F0C
:0E34A900BF08E5D22C8002C22CAF61126F78F2
:0134B70022F2
:0448BF008F5E8D5F1C
:1048C300E55ED394005003024962E55E941540030C
:1048D300024962D22DAF5F125AF27D5F7F051267E4
:1048E300B1AD5EE4FF1267B17D527F041267B17F01
:1048F300F47E01126D4775F020E55E900280123A56
:1049030052AF828583628F63E0F560603DD394008C
:104913004046E56094105040E56025E0F560756120
:1049230001E5602401FFE433FEC3E5619FEE64808B
:10493300F87480985022120FADE0FF120FADA3E080
:10494300FD12663E0561056180D77D1B7F061267F8
:10495300B17D5F7F051267B1C22DAF5F025AF2C20C
:064963002CAF5F126F781B
:01496900222B
:10216D008F5E8D5F8B60E55E640A7074E55FC3946E
:10217D000A40030222DA122310E4FDFF1267B1AD0B
:10218D005F1222E9E55F123A5E21B50121BB022102
:10219D00C10321C70421CD0521D30621D90721DF94
:1021AD000821E509000021EA90052002223490055E
:1021BD002202223490052402223490052602223474
:1021CD0090052802223490052A02223490052C0213
:1021DD00223490052E022234900530804A0222D3FB
:1021ED00E55E64017052E55FD394004006E55F94AF
:1021FD00034006E55F640A703C122310E55FB40AE4
:10220D000A7D0A1222E9900532801CE55FB4010AAD
:10221D007D0B1222F6900534800DE55FB402137D1F
:10222D000C1222F6900536E0FEA3E0FF1265AD021A
:10223D0022E10222D30222DAE55E64026003022269
:10224D00E1E55FD3940050030222DAE55F94075075
:10225D007CD22DAF60125AF27D277F081267B17DB7
:10226D0006E4FF1267B17D14E4FF1267B1E55F2448
:10227D00FE601A14602114602814602F1460362437
:10228D000570437D0112230390053880307D0212C5
:10229D00230390053980267D0312232690053A806D
:1022AD001C7D0412232690053B80127D05122333DD
:1022BD0090053C80087D0612233390053DE0FF7E9E
:1022CD00001265DE800EAF60126CB88007C22CAFB5
:1022DD0060126F78C22DAF60125AF222E4FF1267BE
:1022ED00B17D527F041267B122E4FF1267B17D52B6
:1022FD007F041267B122E4FF1267B17D527F041291
:10230D0067B122D22DAF60125AF27D277F08126776
:10231D00B17D06E4FF1267B122E4FF1267B17D5271
:10232D007F041267B122E4FF1267B17D527F041260
:03233D0067B12263
:044BE8008E638F64E5
:104BEC000564E5647002056314F5828E83E0F56656
:104BFC00607AC3940850757F2C7E01126D47E4F5E2
:104C0C0065E565C395665064856482856383E012AF
:104C1C003A5E4C59004C370A4C3B0B4C410C4C4700
:104C2C000D4C4D0E4C530F00004C5FE4FD802D7D60
:104C3C005F7F0780287D5E7F0680227D0A7F028051
:104C4C001C7D327F0280167D467F0280107D0A7F9C
:104C5C0003800A856482856383E0FDE4FF1267B1FB
:0C4C6C000564E564700205630565809531
:014C78002219
:061F7B008F5E8D5F8B609C
:101F8100C22BE55E640A600302206FE55F123A5ED0
:101F91001FB0011FC3021FD6031FE9041FFC052048
:101FA1001206202807203E082053090000206B124A
:101FB10020A47D011220F2756101756200D22B020D
:101FC100208B1220A47D021220F275610175620836
:101FD100D22B02208B1220C07D031220FF756101DC
:101FE100756210D22B02208B1220C07D041220FFBB
:101FF100756101756218D22B02208B1220DC12212F
:10200100527D05122122756101756220D22B0220B9
:102011008B1220DC1221527D06122122756101757D
:102021006228D22B02208B12210C1221667D07120D
:10203100212F756101756230D22B02208B12210C88
:102041001221667D0812212F756101756238D22B2C
:10205100803812213CE4FDFF1267B17D091221593C
:10206100756101756240D22B8020C22B801CE55E18
:1020710064017016E55F24F6701012213C7D0A128E
:102081002159756101756258D22B302B09AF62AEAF
:1020910061124BE88005AF60126CB8C22DAF6012BF
:0220A1005AF2F1
:1020A30022D22DAF60125AF27D577F021267B17DA3
:1020B30005E4FF1267B1E4FDFF1267B122D22DAF31
:1020C30060125AF27D577F021267B17D05E4FF1259
:1020D30067B1E4FDFF1267B122D22DAF60125AF24D
:1020E3007D577F021267B17D05E4FF1267B122E4D9
:1020F300FF1267B17D527F041267B122E4FF1267BA
:10210300B17D527F041267B122D22DAF60125AF211
:102113007D577F021267B17D05E4FF1267B122E4A8
:10212300FF1267B17D527F041267B122E4FF126789
:10213300B17D527F041267B122D22DAF60125AF2E1
:102143007D577F021267B17D05E4FF1267B122E478
:10215300FDFF1267B122E4FF1267B17D527F0412C3
:0A21630067B122E4FDFF1267B1220C
:1035B8008F72E572D3945940107D5A12369F24A613
:1035C800FD700302369E023699E572D3944F401679
:1035D800E572945A50107D5012369F24B0FD700346
:1035E80002369E023699E572D394454016E57294E8
:1035F8005050107D461236A724BAFD700302369E3D
:10360800023699E572D3943B4012E5729446500C09
:103618007D3C1236A724C4FD607C8075E572D39486
:10362800314012E572943C500C7D321236AF24CEF4
:10363800FD6063805CE572D394274012E572943292
:10364800500C7D281236AF24D8FD604A8043E572BD
:10365800D3941D4016E572942850107D1EE4FF1285
:1036680067B1E57224E2FD602D8026E572D39413DC
:103678004016E572941E50107D14E4FF1267B1E500
:103688007224ECFD60108009E572C394145007ADF4
:1036980072E4FF1267B122E4FF1267B1E57222E417
:0F36A800FF1267B1E57222E4FF1267B1E57222EB
:105AF2008F6AE56A700C302D097F01126FF67FC044
:105B0200801FE56A700C202D097F01126FE37FC0B0
:105B12008026E56AB40112302D0F7F02126FF67FE4
:105B220030120016C22F026A6DE56AB40114202DEC
:105B3200117F02126FE37F30126FA27FC87E0012C4
:035B42006D47228A
:106A49008F69D22D125AF27D607F021267B17D32B1
:106A59007F061267B17D1E7F051267B1C22DAF692E
:046A6900125AF222A9
:106CB8008F69D22D125AF27D607F021267B17D3042
:0D6CC8007F031267B1C22DAF69125AF2228C
:0E6F78008F68302C03026A49AF68126CB82291
:105E8100EF24FE60101460162402701C7F01126F53
:105E9100F67F8080107F02126FF67F2080077F03DC
:105EA100126FF67FA01200167FF47E01126D477506
:105EB1004204E54270FC7F647E00126D477F03124D
:085EC1006FE37FA0126FA22223
:1065DE008E618F627C007D0A1239CCAD07E4FF120A
:1065EE0067B17D5B7F061267B1AE61AF627C007DE5
:1065FE000A1239CCE4FF1267B17D4A7F070267B1F8
:0465AD008E618F620A
:1065B1007C007D3C1239CC1235B87D057F0612670F
:1065C100B1AE61AF627C007D3C1239CCED4C600C08
:0C65D100AF051235B87D4A7F071267B194
:0165DD00229B
:0260D8008D5EDB
:1060DA00120EC5402FEF648094955028120D7178E6
:1060EA0005C333CE33CED8F9120FD6FEE4FD0FEF37
:1060FA00AA0670010E14F5828A83E4F00DBD20EE23
:0B610A00D22C8002C22CAF5E126F7816
:016115002267
:106154008F5E900540E0D394024015D22D125AF27E
:106164007542037F327E00126D47E54270FC801554
:10617400D22DAF5E125AF27D1B7F061267B17D0CE1
:0D6184007F031267B1C22DAF5E125AF222E6
:106E7D007E10900540E4F0A3DEFC7E10D22C126F44
:016E8D00788C
:016E8E0022E1
:106E8F00BF0A02E4FFBD0A02E4FDEF75F00AA42D6C
:026E9F00FF22D0
:106D0F00EFD394094002E4FFEDD394094002E4FD70
:0C6D1F007804EF08800123D8FD4DFF220E
:1040A90007010203040506070707060504030201C1
:1040B90003010A0A030307050303020503020A0AA7
:1040C90004050A0A0104050A0A0A04050A0A020380
:1040D900070A0A03040A0A04024B00020032072EE7
:1040E90003024B0002003202055F000302055F0074
:1040F9000402055F000502055F000604072E082675
:104109000640033204072E08260640025304081EFF
:1041190008260452010008024B00020032072E084B
:104129001E08260452010003072B02350636030731
:104139002B0235063803072B0235072603072B0206
:1041490035025302055F000F02055F001002055F8B
:10415900001102055F001202055F001302055F00EE
:0A41690014080C0A1D020500241BB7
:1053D4007461F0A37420F0A37452F0A37401F0A3D9
:1053E40022A3F0A37461F0A37440F022F0A3740329
:1053F400F0E4A3F0A37410F0A37403F0E4A3F0A307
:10540400227461F0A37441F0A3227461F0A3F0A3A9
:105414007430F0A3227496F0A37432F0A37495F060
:10542400A3741EF0A322F0A37461F0A314F0A37478
:1054340070F0A3E4F022A3F0A37452F0A3223CF58D
:0954440083E0FEEF3395E0FC2249
:10003E007E407FA97C017D507B08125FD67E407F7B
:10004E00B17C017D587B08125FD67E407FB97C0162
:10005E007D007B04125FD67E407FC57C017D087BD0
:10006E0004125FD67E407FC17C017D107B04125F3F
:10007E00D67E407FBD7C017D187B04125FD67E400C
:10008E007FCE7C017D207B05125FD67E407FC97CB2
:10009E00017D287B05125FD67E407FD37C017D30AB
:1000AE007B05125FD67E407FD87C017D387B0412A3
:1000BE005FD67E407FDC7C017D407B04125FD67E66
:1000CE00407FE07C027DA07B09125FD67E407FE9F7
:1000DE007C027DC07B07125FD67E407FF07C027D66
:1000EE00E07B05125FD67E407FF57C037D007B05AD
:1000FE00125FD67E407FFA7C037D207B05125FD691
:10010E007E407FFF7C037D407B05125FD67E417F64
:10011E00047C037D607B09125FD67E417F0D7C03DC
:10012E007D807B09125FD67E417F167C037DA07B8E
:10013E0009125FD67E417F1F7C037DC07B11125F4B
:10014E00D67E417F307C037DE07B07125FD67E41F9
:10015E007F377C047D007B07125FD67E417F3E7C1D
:10016E00047D207B07125FD67E417F457C047D4057
:10017E007B07125FD67E417F4C7C047D607B05122F
:10018E005FD67E417F517C047D807B05125FD67EDB
:10019E00417F567C047DA07B05125FD67E417F5B3E
:1001AE007C047DC07B05125FD67E417F607C047D22
:1001BE00E07B05125FD67E417F657C057D007B0569
:1001CE00125FD67E417F6A7C057D407B09125FD629
:1001DE009000297417F07F031264E19000287419BF
:1001EE00F090002074B1F09000217491F0900022F4
:1001FE007403F0900023747FF090002404F09000BC
:10020E00257403F0E4900026F0900027F090003063
:10021E0074091253F07415F0A37403F0A37415123D
:10022E0053F07409F0A37403F0E4FFEFFD3395E08F
:10023E00FC74302DF582740012544274102DF58228
:10024E0074003CF583EEF00FBF08E0E4FFEFFD33E2
:10025E0095E0FC74382DF582740012544274182DFA
:10026E00F58274003CF583EEF00FBF08E090052098
:10027E00E4F0A374B4F0900522E4F0A374B4F0900B
:10028E0005247401F0A374E0F0900526E4F0A37445
:10029E0078F09005287402F0A37458F090052AE4C3
:1002AE00F0A3743CF090052C7402F0A37458F07413
:1002BE000790052EF0A3F0900530F0A3F0900532D4
:1002CE00F0A3F0900534F0A3F0900536E4F0A3749B
:1002DE003CF0900538740AF09005397428F09005BA
:1002EE003A7405F090053B740AF090053CF09005C9
:1002FE003D7428F09000A47401F0900B607415F01A
:10030E00A37411F09000A57401F0900B807415F099
:10031E00A37410F09000A67401F0900BA07415F069
:10032E00A37421F09000A77401F0900BC07415F027
:10033E00A37420F09000A87401F0900BE07415F0F7
:10034E00A37431F09000A97401F0900C007415F0B4
:10035E00A37430F09000AA7401F0900C207415F084
:10036E00A37441F09000AB7401F0900C407415F042
:10037E00A37440F09000AC7401F0900C60745312B2
:10038E0053DE74361253DE7438F0A3E4F0A37453C4
:10039E00F0A3E4F09000AD04F0900C80745312536F
:1003AE00DE7434F0A37421F0A37453F0A3E4F09040
:1003BE0000AF04F0900CC01253DC7430F0740312D2
:1003CE00543AE4F09000B004F0900CE01253DC7458
:1003DE0030F0740412543AE4F09000B104F0900D31
:1003EE00001253D474321253DE7452F0A37420F000
:1003FE009000B27401F0900D201253D47432F0A319
:10040E00740212543B7420F09000B37401F0900DFE
:10041E004074531253DE7433F0A3E4F09000B4042E
:10042E00F0900D601254057430F074021253E59082
:10043E0000B57401F0900D801254057430F07405FF
:10044E001253E59000B67401F0900DA0125405748D
:10045E0030F0A374061253E69000B77401F0900DBD
:10046E00C01254051254197498F0A3744B1253E62B
:10047E009000B87401F0900DE012540512541974E6
:10048E0093F0A374181253E69000B97401F0900E15
:10049E00001254057430F0A374131253E6A3747053
:1004AE00F0A37402F09000BA14F0900E2012540EC5
:1004BE007412F0A374701253DE7461F0A314F090F2
:1004CE0000BB7401F0900E4012540E741112542A97
:1004DE009000BC04F07461900E60125410741412EB
:1004EE00542A9000D104F09011001254057492F029
:1004FE00A3744BF0A37490F0A37402F0A37490F065
:10050E00A37432F07499A3F0A3F0A374601253DEB7
:10051E0074911253DE7491F0A3E41253E690000F1F
:10052E007401F0125EC97F01126FF67F4012001641
:10053E007D2F7F071267B17D0C7F031267B17D326D
:0C054E007F061267B17D1E7F051267B1A9
:01055A00227E
:0A5FD6008E5A8F5B8C5C8D5D8B5E34
:105FE000E4F9C3E55E6480F8E96480985028E9FF2D
:105FF0003395E0FEE55B2FF582E55A3EF583E493A9
:10600000FFE9FD3395E0FCE55D2DF582E55C3CF5AF
:0660100083EFF00980CCD3
:016016002267
:10575400AF6AEF3395E0FEE56975F008A42428F5F7
:1057640082E43400F583E5822FF582E5833EF583F8
:10577400E0FFE56AFD3395E0FC22AB66AD65AF64FE
:10578400223EF583E0FD74B82FF582741D3EF58347
:10579400EDF0056AE56A22EF3395E0FEEF25E0FFC0
:1057A400EE33FE22A2E0CE13CE13223CF583EFF0BB
:0557B400056AE56A2210
:045C7A008C5B8D5C56
:105C7E00EF6043D201D202D20CE4F55D855C8285E1
:105C8E005B83E0FEA3E04E6027AF5D12579BE55CA1
:105C9E002FF582E55B3EF583E0FEA3E0FF12453271
:105CAE00922920290B055DC3E55D6480949040CC5C
:065CBE00C201C202C20C8B
:015CC40022BD
:045CC5008C608D6101
:105CC900EF6043D201D202D20CE4F562856182858C
:105CD9006083E0FEA3E04E6027AF6212579BE56147
:105CE9002FF582E5603EF583E0FEA3E0FF12453221
:105CF900922D202D0B0562C3E5626480949040CCFF
:065D0900C201C202C20C3F
:015D0F002271
:04453200AD07AC061F
:10453600C22E780CEF0880031257A8D8FB540FF54B
:10454600637808AF05AE04EF0880031257A8D8FBBE
:10455600540FF5647804AF05AE04EF0880031257D4
:10456600A8D8FB540FF565ED540FF566E563607149
:10457600B4010812577E123D348066E563B4020822
:1045860012577E126C238059E563B4030812577ED6
:104596001238AA804CE563B4040812577E126BC425
:1045A600803FE563B4050812577E1224FA8032E58F
:1045B60063B4060812577E1212698025E563B407B4
:1045C6000812577E12525E8018E563B40808125727
:1045D6007E12598E800BE563B4090612577E126966
:0345E600DBA22E27
:0145E90022AF
:103D34008F678D688B69E567B40113900020E0FFFD
:103D4400125A44900020EFF0FD7F20023DF1E56718
:103D5400B40211900021123DF7900021EFF0FD7F95
:103D640021023DF1E567B40311900022123DF79062
:103D74000022EFF0FD7F22023DF1E567B4041090CC
:103D84000023123E01900023EFF0FD7F23805EE5C7
:103D940067B40516900024123E01900024EFF0FD54
:103DA4007F247E0012647602660EE567B4061090E6
:103DB4000025123E0B900025EFF0FD7F25802EE5B7
:103DC40067B40710900026123E0B900026EFF0FD1A
:103DD4007F268019E567B40819900027E0FFAB69D6
:103DE400AD68125A44900027EFF0FD7F277E001241
:103DF400647622E0FFAB69AD68125A4422E0FFAB5F
:103E040069AD68125A4422E0FFAB69AD68125A44A6
:013E1400228B
:105A4400D22FAC07BD01047E018033BD02047E0267
:105A5400802CBD03047E048025BD04047E08801EC2
:105A6400BD05047E108017BD06047E208010BD078E
:105A7400047E408009BD08047E808002C22FBB01E1
:105A840005EE4204800BEB7006EEF452048002C271
:075A94002F302F03AF0422A5
:015A9B0022E8
:026C23008B677D
:106C2500C22FEF7016ED7013E5677003025D5BE52B
:0B6C350067B40107787FE6FF125B9553
:016C40002231
:0638AA008F678D688B6939
:1038B000E5677007123990E4FD801AE567B40107E7
:1038C0001239907D01800EE567B4020CAD69AF68D6
:1038D000126F867D0202504FE567B40306124173F2
:1038E000C21E22E567B40415AD69AF681265498F41
:1038F00043754205E542700302398F80F7E567643E
:10390000067017E5687013F56A12575474102DF598
:103910008274001257AFB408F022E567640770178D
:10392000E5687013F56A12575474182DF582740007
:103930001257AFB408F022E56764087027E5687095
:1039400023E569701FF56AAF6AEF3395E0FE7410E6
:103950002FF5827400125785B408EC754201E542D8
:10396000602D80FAE56764097025E5687021E569D6
:10397000701DF56AAF6AEF3395E0FE74182FF5827B
:0F3980007400125785B408EC754201E54270FCE3
:09398F0022AD69AF68126F8622B7
:106BC4008F67AE03AF05E567D394004012E5679481
:106BD40007500CAD06126F86AD07AF671268052229
:1024FA008F678D688B69E5677018E5687014E56900
:10250A0070057F01126FA2E569640160030226A7C4
:10251A008043E567701CE568B40117E56970057FBB
:10252A0004126FA2E569640160030226A77F040210
:10253A0026A4E5677029E56864027023E5697005D9
:10254A007F05126FA2E569640160030226A7900065
:10255A000FE0B403057F010226A47F050226A4E545
:10256A0067B4011BE5687017E56970057F02126F91
:10257A00A2E569640160030226A77F020226A4E598
:10258A0067B4011CE568B40117E56970057F081294
:10259A006FA2E569640160030226A77F080226A4E8
:1025AA00E56764017029E56864027023E5697005CE
:1025BA007F0A126FA2E569640160030226A79000F0
:1025CA000FE0B403057F020226A47F0A0226A4E5CF
:1025DA0067B4021BE5687017E56970057F40126FE2
:1025EA00A2E569640160030226A77F400226A4E5EA
:1025FA0067B4021CE568B40117E56970057F10121B
:10260A006FA2E569640160030226A77F100226A46F
:10261A00E56764027024E5686402701EE569700566
:10262A007F50126FA2E5696401707290000FE0B4E6
:10263A0003047F4080647F508060E567B40317E538
:10264A00687013E56970057F80126FA2E5696401FD
:10265A00704B7F808044E567B40318E568B40113C2
:10266A00E56970057F20126FA2E5696401702E7F0B
:10267A00208027E56764037024E5686402701EE51C
:10268A006970057FA0126FA2E569B4011090000F6E
:0E269A00E0B403047F8080027FA012001622AD
:101269008F678D688B69E5677017AD69AF68126F15
:10127900868E348F35D3E5359400E534940050F5E6
:1012890022E567B4011BE568B40116E5697007C278
:10129900307F01122ECAE569640160030214D68009
:1012A90058E5676401702BE56864027025E569708B
:1012B90007C2307F02122ECAE56964016003021475
:1012C900D690000FE0640370030214D6D2307F0277
:1012D9008031E5676401702EE56864037028E5696B
:1012E9007007C2307F03122ECAE5696401600302E8
:1012F90014D690000FE0B40306D2307F018004D2E7
:10130900307F03022ECAE5676401702DE568640425
:101319007027E569700CC2307F01122ECA7F401216
:101329006FA2E569640160030214D6D2307F01120D
:101339002ECA7F40120016807CE5676401703AE589
:101349006864057034E569700CC2307F02122ECAD8
:101359007F10126FA2E569640160030214D6900040
:101369000FE0640370030214D6D2307F02122ECA32
:101379007F10120016D22F803EE5676401703BE5AD
:101389006864067035E569700CC2307F03122ECA95
:101399007F50126FA2E569640160030214D6D2304E
:1013A9007F03122ECA90000FE0B403047F4080022D
:1013B9007F50120016C22F026A6DE5676402702918
:1013C900E56864017023E56970057F100214BDE5C5
:1013D90069B401057F100214C7E56964026003025C
:1013E90014D6D22F7F010214D3E56764027029E570
:1013F9006864027023E56970057F200214BDE56900
:10140900B401057F200214C7E56964026003021470
:10141900D6D22F7F020214D3E56764027029E568EA
:1014290064037023E56970057F400214BDE569B462
:1014390001057F400214C7E569640260030214D6FE
:10144900D22F7F030214D3E56764027023E5686431
:1014590004701DE56970047F808059E569B4010451
:101469007F80805AE56964027063D22F7F04805AB5
:10147900E56764027023E5686405701DE569700419
:101489007F048030E569B401047F048031E5696433
:1014990002703AD22F7F058031E5676402702EE52C
:1014A90068640670287D017F07124F40401FE56977
:1014B90070057F08026FE3E569B401057F08026FD3
:0E14C900F6E569B40207D22F7F06122992229F
:06525E008F678D688B696B
:10526400E567703BE5687037E569700690000F04E8
:105274008021E569B4010A90000F7402F0D22F80F6
:1052840047E56964027041C21E7FFF126FA290005D
:105294000F7403F0C2307F02122ECAD22F8029E588
:1052A4006764017023E568701F7D077F05124F4016
:1052B4005016E569700BC200C2307F03122ECA80FB
:1052C40007E569B40102D200302F0C90000FE0FD15
:0752D4007F0F7E00126476DB
:0152DB0022B0
:10598E008F678D688B69E567700C1259D2749F2FE3
:10599E00F58274008019E567B4010C1259D2749F18
:1059AE002FF58274008016E567B402091259DA3EAB
:1059BE00F583E4F022E567B403091259DA3EF58364
:1059CE007401F022AD69AF68126F8622AD69AF68BF
:0B59DE00126F86746F2FF58274002298
:0269DB008F67C4
:1069DD00AF057804EF08800123D8FD4BF568E56716
:1069ED00B40908E568B49903024FC8AD68AF6712E2
:0269FD00663EF4
:0169FF002275
:0D6F8600EF75F00AA47C002DFFEC35F0FE45
:016F930022DB
:046805008F688D69A2
:10680900C3E569648094E4501BE4F56AC3E56964EF
:1068190080F8E56A648098500BC22FAF68122992FC
:04682900056A80E894
:01682D002248
:0D6F9400C296007F0512694512657BD296FA
:016FA10022CD
:106E2B00126F94EF20E0F9C296007F06126945C2FB
:066E3B00B60000D2962211
:106E4100126F94EF20E0F9C296007F04126945C2E7
:066E5100B60000D29622FB
:046116008E608F61A7
:10611A00AE04AF058E638F64C296007F0312694591
:10612A00E560FF126945AF61126945E4F5621265DF
:10613A007BE5642562F582E43563F583EFF0056259
:09614A00E562C3942040E7D296FF
:016153002229
:085D10008E658F668C678D68BB
:105D1800126F94EF20E0F985656A85666BC296007C
:105D28007F02126945E567FF126945AF6812694548
:105D3800E4F569E56B2569F582E4356AF583E0FFEA
:105D48001269450569E569C3942040E7C2B60000B9
:025D5800D296E1
:015D5A002226
:0A56EE008E5A8F5B8C5C8D5D8B5E25
:1056F800C2AF126E2B126F94EF20E0F9855C6085C3
:105708005D61C296007F02126945E55AFF1269453C
:10571800AF5B126945E4F55FAF5EEF3395E0FEC31A
:10572800E55F9FEE6480F87480985014E561255F0A
:10573800F582E43560F583E0FF126945055F80D89E
:0B574800C2B60000D296126E41D2AF34
:015753002233
:106476008E6B8F6C8D6DC2AF126E2B126F94EF20E8
:10648600E0F9C296007F02126945E56BFF12694585
:10649600AF6C126945AF6D126945C2B60000D2965F
:0664A600126E41D2AF228C
:10619100C2AFE4F55BF55CF55DF55EF55FF55AAE12
:1061A1005EAF5FAC5BAD5C1261167420255CF55C83
:1061B100E4355BF55B7420255FF55FE4355EF55EE4
:0B61C100055AE55AC3948940D6D2AFBE
:0161CC0022B0
:105EC900C2AF756200756300756400E4F560F56141
:105ED900F55F126E2BAE63AF64AC60AD61125D10FD
:105EE90074202561F561E43560F56074202564F559
:105EF90064E43563F563055FE55FC3948940D312B4
:045F09006E41D2AF64
:015F0D002271
:105818000500050105030507050F051F051E051CE5
:10582800051805100201040E040A03060101040B01
:105838000304040F020304010302040D0200020220
:105848000300040904040305030701000303040714
:10585800030104060402040C0516051500000615CC
:0E586800062A060C06380633061E0612061720
:104D99002430F58274003EF583EDFF3395E0FEE59E
:104DA900822FF582E5833EF583E0FFEDFB3395E045
:104DB900FA22AF41126945C293126FEDD293D2AF75
:104DC900223EF583E0FC74B82FF582741D3EF5830D
:104DD900ECF00D221528E528D394002225E02418AB
:104DE900F582E43458F583E49322E4F57BD20EC2CC
:104DF90027C21DC21A227FA0126FA2E4F542C21E69
:104E090022126FEDD2B67801EF0822122C44D2CAD1
:0F4E1900D20ED22722ECFF3395E0FEEF78032272
:10423900200E2F900540E004F576D36480948150D8
:10424900030242F9D3E5766480948F400375760FB3
:10425900900029E0FF122C4490002AE0F575124DD8
:10426900F322301A58302712124DDD40030242F969
:10427900C2CAC227D21D85752822301D0A124DDDFA
:10428900506EC227C21D22AF791579EF700BC21A81
:10429900E57525E0F528D21D22E57A30E00585751A
:1042A900288008E57575F003A4F528AF7A7801EF41
:1042B90008800103D8FDF57AD227D2CA22D576081B
:1042C900C20EE4F542C21E22057B7440257BF582AD
:1042D900E43405F583E0124DE5540FF57974019343
:1042E900F57A700AD21DE57525E025E0F528D21A80
:0142F90022A2
:1052DC00200E12900029E0FF122C4490002AE0F5D9
:1052EC0077124DF322301A5130270F124DDD505DDD
:1052FC00C2CAC227D21D85772822301D0A124DDD65
:10530C00504BC227C21D22AF791579EF7007C21A14
:10531C00C20EF54222E57A30E0058577288008E553
:10532C007775F003A4F528AF7A7801EF08800103B4
:10533C00D8FDF57AD227D2CA22E543124DE5FA748C
:0D534C000193FBEA540FF579EBF57AD21AC4
:015359002231
:10657B00E4F56FD297F56EC2B6126FEDAF6F78017F
:10658B00EF08800123D8FDF56F309703436F01129D
:10659B006FEDD2B6056EC3E56E6480948840D8AFBC
:0165AB006F80
:0165AC0022CC
:096FED0000000000000000002279
:10675A00C2B7E4FEC2B6126FEDEF30E704D2B580DD
:10676A0002C2B5124E0A800123D8FDFF126FED0E48
:0B677A00BE08E1C2B6D2B7D2B6D2B55D
:0167850022F1
:0D001600C2AFEF4227AF2712675AD2AF22C8
:0E6FA200C2AFEFF45227AF2712675AD2AF22C8
:10694500E4FEC2B6126FEDEF30E704D2B58002C2A5
:10695500B5124E0A800123D8FDFF126FED0EBE0859
:05696500E1D2B6D2B53D
:01696A00220A
:096FF600C2AFEF4241124DBB2273
:0A6FE300C2AFEFF45241124DBB2281
:102C4400EF123A5E2CAC012CB3022CBA032CC10453
:102C54002CC8052CCF062CD6072CDD082CE4092C17
:102C6400EB0A2CF20B2CF90C2D000D2D070E2D0E5A
:102C74000F2D15102D1C112D23122D2A132D311457
:102C84002D38152D3F162D46172D4D182D54192D61
:102C94005B1A2D621B2D691C2D6B1D2D721E2D7947
:102CA4001F2D802000002D6975CB8E75CAC6227534
:102CB400CB9575CA772275CB9B75CA692275CBA053
:102CC40075CABA2275CBA675CA332275CBAB75CA41
:102CD400632275CBB075CA022275CBB475CAA32220
:102CE40075CBB875CAFA2275CBBC75CAD82275CB18
:102CF400C075CAA82275CBC475CA362275CBC775F0
:102D0400CA862275CBCA75CABC2275CBCD75CAB426
:102D14002275CBD075CA762275CBD375CA3022758D
:102D2400CBD575CAB22275CBD875CA132275CBDA46
:102D340075CA522275CBDC75CA7D2275CBDD75CA86
:102D44006E2275CBE075CA542275CBE275CA1B227C
:102D540075CBE375CAC32275CBE575CA5E2275CB04
:102D6400E675CADA22801C75CBE875CA902275CB49
:102D7400EA75CAD92275CBEC75CA092275CBED75F3
:0A2D8400CA292275CBE875CA412266
:10002600C3EF648094A15008EF25E025E0F528226F
:04003600E4F52822A3
:0237B3008F5A2B
:1037B500900118E0FFE55A7006E545D39F5012E5E4
:1037C5005A640160030238A9E546D39F50030238C5
:1037D500A9E55A7018C3E5459FF55D74602FF5821C
:1037E500E4341EAD82F55E8D5F7F40801BE55AB4E3
:1037F5000119C3E5469FF55D74B02FF582E4341ECB
:10380500AF82F55E8F5F7F101200167FF47E011286
:103815006D477D207F051267B17D1A7F081267B15C
:103825007FC87E00126D47E4F55BE55BC3955D508F
:1038350061055FE55FAE5E7002055E14F5828E83FD
:10384500E0F55C123A5E38860038640A38680B3851
:103855006E0C38740D387A0E38800F0000388CE401
:10386500FD80277D5F7F0780227D5E7F06801C7D32
:103875000A7F0280167D327F0280107D467F02809E
:103885000A7D0A7F038004AD5CE4FF1267B1055B26
:103895008098E55A70047F408007E55AB401057F9A
:0438A50010126FA2EC
:0138A90022FC
:10515B00200E10754406901DB8E06003D20E22E4B9
:10516B00F54222E528D394004003152822C2CA1524
:10517B0044E54414603D14603214601D1460151432
:10518B007049901DB8E0FF7003F54222122C449039
:10519B001DB9802F901DBA8015901DBBE0FF7003C9
:1051AB00F54222122C44901DBC8018901DBDE0FFCF
:1051BB00020026901DBEE0FF7003F54222122C4424
:1051CB00901DBFE0FF120026D2CA22E4F542C2CAEC
:0351DB00C20E22DF
:10672C00900028E0FF6026200E07124E14752814E6
:10673C0022E528D394004003152822202708D2CA2A
:0E674C00752814D22722C2CA75287DC22722C2
:1066CE00200E0C7F1C124E1475286475783C22E542
:1066DE0028D394004003152822AF781578D3EF64A1
:0E66EE00809480400475286422C20EE4F542B8
:0166FC00227B
:1063D300E54214601C14601C14601F1460221460D6
:1063E3002224057021C2CAC20EC227C21DE4F5448D
:1063F3002202515B12672CD21E22124239D21E2274
:076403000266CE1252DC22FA
:1064E100BF010790002A7418F022BF020790002A0A
:1064F1007412F022BF030590002A8014BF04079094
:10650100002A740BF02290002ABF05047409F022BE
:04651100740CF022F4
:0250D500AC0726
:1050D700C3EC64809480404AEC64809488504320F9
:1050E7002B21E4FD124E1EC333CE33CED8F9124D19
:1050F7009974102BF58274003AF583EFF00DBD0813
:10510700E3801FE4FD124E1EC333CE33CED8F9120F
:105117004D9974182BF58274003AF583EFF00DBDA5
:1051270008E3202B16E4FDEDFF3395E0FE74102F06
:10513700F5827400124DCABD08ED22302B15E4FD2F
:10514700EDFF3395E0FE74182FF5827400124DCAF7
:03515700BD08EDA3
:01515A002232
:104FC8007D3F7F091267B17D507F081267B19070ED
:104FD8001F1250467D5B7F061267B19070201250F9
:104FE80046907021E493FDE4FF1267B1907022E4CB
:104FF80093123A5E501841501C42502043502644A8
:10500800502C45503246503847503E4800005045D5
:105018007D0A80067D3280027D467F02801C7D0AE3
:105028007F0380167D287F0380107D467F03800ADA
:105038007D0A7F0480047D287F041267B122E493EF
:07504800FDE4FF1267B12235
:106058008F5BE55B7005D22DFF8009E55BB4010716
:10606800D22D7F01125AF27D4B7F021267B17D0259
:10607800E4FF1267B17D32E4FF1267B1124FC8E541
:106088005B70028005E55BB401057F40126FA222B8
:103E1500A209300501B350307D017F04124F405097
:103E25002320050E30090B9000A4E0FF7C0B7D607C
:103E3500800F30050F20090C9000A5E0FF7C0B7D5D
:103E450080125CC5A2099205A20A300601B3503062
:103E55007D027F04124F40502320060E300A0B903E
:103E650000A6E0FF7C0B7DA0800F30060F200A0C1A
:103E75009000A7E0FF7C0B7DC0125CC5A20A9206EC
:103E8500A20B300701B350307D037F04124F405021
:103E95002320070E300B0B9000A8E0FF7C0B7DE084
:103EA500800F30070F200B0C9000A9E0FF7C0C7DE4
:103EB50000125CC5A20B9207A20D300801B3503069
:103EC5007D047F04124F40502320080E300D0B90C7
:103ED50000AAE0FF7C0C7D20800F30080F200D0C20
:103EE5009000ABE0FF7C0C7D40125CC5A20D9208F2
:013EF50022AA
:10660E00534103900024E0FE543FFF7804088001BC
:10661E0023D8FD54F0FFEE30E4034307049000242A
:0F662E00E030E503430708EF4241C2AF124DBB16
:01663D00223A
:022992008F6B49
:10299400302F05756CF48003756C64E56B6401700D
:1029A40029AF417803EF08800123D8FD3392307FAB
:1029B4001020300B122AAE7F10126FE3022AA612E7
:1029C4002AB97F10126FF6022AA6E56B64027028FA
:1029D400AF417802EF08800123D8FD3392307F2085
:1029E40020300A122AAE7F20126FE38008122AB91F
:1029F4007F20126FF6022AA6E56B64037028AF41AC
:102A04007801EF08800123D8FD3392307F402030D5
:102A14000A122AC47F40126FE38008122ACF7F4033
:102A2400126FF6022AA6E56B6404701EE541339228
:102A3400307F8020300A122AC47F80126FE380081E
:102A4400122ACF7F80126FF68058E56B64057027D9
:102A5400AF417805EF08800123D8FD3392307F041D
:102A640020300A122ADA7F04126FE38008122AE562
:102A74007F04126FF6802BE56B6406702CAF4178EF
:102A840004EF08800123D8FD3392307F0820300AF8
:102A9400122ADA7F08126FE38008122AE57F0812EF
:092AA4006FF6AF6C7E00126D4765
:102AAD0022126FF6AF6C7E00126D4722126FE3AFEC
:102ABD006C7E00126D4722126FF6AF6C7E00126DA8
:102ACD004722126FE3AF6C7E00126D4722126FF634
:102ADD00AF6C7E00126D4722126FE3AF6C7E001259
:032AED006D472210
:105E3800900024E030E0057F10126FF6900024E017
:105E480030E1057F20126FF6900024E030E2057FF4
:105E580040126FF6900024E030E3057F80126FF661
:105E6800900024E030E4057F04126FF6900024E0EF
:095E780030E5057F08126FF622E7
:106D980030030A124DFFC203C211C21E2230040979
:0A6DA800124DFFC204C213C21E22E6
:10663E008F708D71E570B4011FE5717003125D5B93
:10664E00E571B40107787FE6FF125B95E571B43210
:10665E000E7FF47E01026D47AD71AF701267B122ED
:1067B100EFFEEDFF1280008E2D8F2E1254C27574E4
:1067C10032AF741574EFD39400400EE4F573E573A2
:0967D100C3943A50EC057380F505
:0167DA00229C
:1054C200D2A8AFA875A881C214852E82852D83E447
:1054D20093C4540FFE4306F08E80C284D28500C26C
:1054E200870000D287007580FF7580FEC284C28566
:1054F20000C2870000D287007580FFD2147D407CF5
:105502001FE4FE30B40D0EBE32F9ED1D70011CED2C
:105512004C70EE7C1F7D40E4FE20B40D0EBE32F9CD
:10552200ED1D70011CED4C70EE8FA8C2A87F0A7EA3
:0455320000126D47AF
:015536002252
:1067DB007580FDC284C28500C28700000000D2878D
:1067EB00007580FF7F0A7E00126D477F997E09122C
:0A67FB0080008E2D8F2E1254C22252
:1042FA00D284D285C286A2809217A2819220A282FB
:10430A009218A2839221D2862001537D027F011244
:10431A004F4040137D037F01124F40400A30170778
:10432A00301932D22480377D027F01124F40500F5C
:10433A0030170C302009301904D224802180167DD0
:10434A00037F01124F40501220170330200C3019FE
:10435A0004D224800912687F8004C219C224200270
:10436A004E7D027F02124F4040127D037F02124FA0
:10437A00404009301806301B2FD225227D027F02C9
:10438A00124F40500E30180B302108301B03D22533
:10439A002280157D037F02124F40500F20180330F0
:1043AA002109301B03D225220268A7C21BC225227B
:10687F00753D1E753E60E4FFE53E2FF582E4353D24
:10688F00F583E4F00FBF50F0753D1E753E60E4F5E3
:07689F0045C226C211D21907
:0168A60022CF
:1068A700753F1E7540B0E4FFE5402FF582E4353FA4
:1068B700F583E4F00FBF10F0753F1E7540B0E4F5A7
:0768C70046C228C213D21BD8
:0168CE0022A7
:106CD500C284D285C286A2809209A281920AA2822A
:0D6CE500920BA283920DD286D284D285221A
:10620900E57D2560F582E4357CF5832274FF123A39
:1062190034E4FBFAF9F8C3023A21057E7480257D3E
:10622900F57DE4357CF57C22F582E4341DF5832285
:0B623900757E01757C00757D20E4225D
:1043BA007D027F07124F4050057F04126FE3C22926
:1043CA00D223E4F5427FE87E03126D47C298C2AF5A
:1043DA00C2307F03122ECA755E7F755D96755C9832
:1043EA00755B00785B126215504430983E120006E5
:1043FA00126EF9EF14601824F0602624C1600B24B1
:10440A00F670287F0612700880211262F3801C7FE2
:10441A0006127008126AB312660E125EC9D2298099
:10442A000A7F06127008125B45D2293029B5E47852
:10443A0084F6D2307F01122ECA7F40120016C22F94
:10444A00126A6D7D467F021267B17D1E7F07126771
:10445A00B17D147F081267B17D327F031267B1C242
:0D446A00307F03122ECA7FFF126FA2C22303
:014477002222
:105B4500126239F55F7F02127008E57E2402F56165
:105B5500AF7E127008E4F560126209E0FF1270086A
:105B6500126209E02561F5610560E560C394804036
:105B7500E7AF611270087F03127008127010EF64AE
:0F5B850015600C126223055FE55FC3942240B6E2
:015B940022EE
:106AB300126239F55F12651550077F061270088060
:106AC300057F15027008126223055FE55FC39422F8
:026AD30040E39E
:016AD500229E
:10651500E4F56012701074D02560126231EFF00559
:1065250060E560C3948440EB126ED7901E52E0B5CF
:106535000710AE7CAF7DBE0504BF200100126D2B98
:03654500D322C39B
:016548002230
:106D2B00E4FF74D22FF582E4341DF583E0FEE57D9C
:0B6D3B002F12620DEEF0000FBF80E78A
:016D4600222A
:106ED700E4FFFE74D02E126231E02FFF0EBE82F364
:016EE7002288
:1062F300E4F55FF5657564E0756393756204F561B4
:10630300786112621550213098F61200068F60E50D
:106313006064046013AF65056574D02F126231E5C4
:0863230060F0255FF55F80D8F2
:01632B00224F
:04000600AF99C29854
:01000A0022D3
:087008003099FDC2998F992215
:077010003098FDAF99C29812
:017017002256
:106DE5000C0102030405060708090A0B0C0102033E
:086DF5000405060708090A0B5A
:10682E00AF5FEF3395E0FE75F007EF123A52EE755B
:10683E00F007A42583F583E0227882E6FF126DCC63
:09684E00EF22C295D297D2AF22CD
:10696B00C22CC2AF1270187F83126DFD126BE41232
:10697B0068507883E66F600B125F94302B051260C2
:05698B0098922CA22CE3
:0169900022E4
:106098007983E778866660367883E6FF7886F6EF58
:1060A8007013E552C3940A500C7D077F04124F40C9
:1060B8005003125F0E7D057F04124F405010E541DA
:1060C80054036005123FD6D322123FD6C322C322FF
:103FD600E4F55F900A5012682E700302409A900A28
:103FE600511268356016788066600302409A900A1E
:103FF6005212682E788766600302409AAF5FEF33ED
:1040060095E0FE900A53126835FF787FE6FEEF6E64
:104016006020EF601DB4080BEED394014005EE94CA
:1040260007400FEF6409706CEE64016005EE6407EB
:104036007062AF5FEF3395E0FE900A54126835FF69
:10404600F46006EF788266704BE55FFD3395E0FC21
:10405600900A5575F007ED123A52EC12683D7883D6
:10406600667031D201D20274BD2DF58274003CF522
:1040760083E0FFC007EDAE047805C333CE33CED858
:10408600F92480F582740E3EAD82FCD007125CC521
:10409600C201C202055FC3E55F64809493500302C8
:0240A6003FD900
:0140A80022F5
:105F0E007D087F04124F40500D7882E6FF126DCC53
:105F1E00EFC39407402CD2307F01122ECA7F40125D
:105F2E000016C22F126A6DD201D202E4FD7F0A1250
:105F3E00504FC201C2027F50126FA2C2307F0112B7
:035F4E002ECA2236
:105F9400C2AF1270187FBF126DFD126BE47883A636
:105FA40007126BE47883A607126BE47882A60712C3
:105FB4006BE47887A607126BE47880A607126BE47B
:105FC400787FA607126BE47881A60712701812680E
:025FD400502259
:1059E900C2AF1270187F8E125A387F90126DFD7FE8
:1059F900A7126DFD1270187FBE126DFDE4FF126DC6
:105A0900FD7883E6FF126DFD7882E6FF126DFD7861
:105A190087E6FF126DFD7880E6FF126DFD787FE65F
:105A2900FF126DFD7881E6FF125A38126850221272
:0B5A39006DFDE4FF126DFD12701822DD
:105B95008F72E572B401047D63803EE572B402063E
:105BA5007D087F068035E572B403067D317F088068
:105BB5002AE572B404067D617F08801FE572B4058D
:105BC500067D257F088014E572B406067D597F039E
:0F5BD5008009E572B407077D487F071267B12288
:026DCC00AE0710
:106DCE00EE54F0FF780408800103D8FD75F00AA494
:066DDE00FFEE540F2FFF31
:016DE400228C
:105D5B00126847906DE593FF1235B8788312684946
:105D6B00601B7883126849C3940A50077D327F0603
:105D7B001267B17883E6FF126DCC1235B812684703
:105D8B00C3940C50067D0A7F0280047D507F06125F
:0A5D9B0067B17D507F051267B12249
:105A9C007FF47E01126D477D097F061267B1788015
:105AAC00125AE27D0E7F031267B17D357F061267B5
:105ABC00B17D097F061267B17887125AE27D1E7F8D
:105ACC00091267B17D1E7F071267B17881E6FF125C
:105ADC006DCC1235B822E6FF126DCC1235B87FF4BE
:065AEC007E01126D47224D
:07701800C2B6C295D2952219
:106DFD00E4FEC297EF30E002D297C2B6D2B6EFC32F
:066E0D0013FF0EBE08ECAD
:016E1300225C
:106BE400E4FFD297FED2B6C2B6A297E433C43333DD
:0F6BF400335480FDEFC313FFED42070EBE08E6DA
:016C0300226E
:10593100EF3395E0FE74702FF58274003EF583E03D
:10594100FF22AF5AEF3395E0FEEF222460F5827417
:10595100013EAD82FCD22922900520E0F547A3E06B
:10596100F548222450F58274053EAD82FC22900058
:10597100BAE0FF7C0E7D2022D222D201E4FF22C2B6
:0D59810001C2227F1922D222D2307F0222E1
:10283100E5527008126FCC8F5202292CE552B40573
:10284100081245EA8F5202292CE552B40B08126D89
:10285100628F5202292CE552B40A08125DA58F52EB
:1028610002292CE552B40F08125F518F5202292C14
:10287100E552B414081223408F5202292CE552B4B8
:102881001908126C418F5202292CE552B41E08120C
:102891006B1C8F5202292CE552B42308126B828FD4
:1028A1005202292CE552B42807126FB08F52807B57
:1028B100E552B42D071268F78F52806FE552B4329A
:1028C1000712632C8F528063E552B43E07126C5F8E
:1028D1008F528057E552B43C07126EA18F52804B44
:1028E100E552B43307126B608F52803FE552B44119
:1028F10007126F2A8F528033E552B44C07126F3A98
:102901008F528027E552B44407126F4A8F52801BC1
:10291100E552B437071257B98F52800FE552B439D7
:10292100071255378F528003E4F552E553700612B2
:10293100000E8F5322E553B40506126FFF8F532209
:10294100E553B40A06126F5A8F5322E553B40F06AA
:10295100126F698F5322E553B41406123C518F5301
:1029610022E553B43D06126C7D8F5322E553B43FEB
:102971000612666E8F5322E553B443061268CF8F59
:102981005322E553B44D06126BA38F5322E4F55342
:012991002223
:0D6FCC0090052AE0F52BA3E0F52C7F0522AF
:1045EA00302414201011C21C7D047F01124F405048
:1045FA00037F0B227F0A227F0812640A50061247A1
:10460A00557F0022202408301005C2107F05227D24
:10461A00057F06124F40501EE53945387018900044
:10462A00B5E0FF7C0D7D80125CC590052EE0F53863
:10463A00A3E0F53980517D067F06124F40501EE5F2
:10464A003C453B70189000B6E0FF7C0D7DA0125CE3
:10465A00C5900530E0F53BA3E0F53C802A7D077F55
:10466A0005124F40500B300008E52C452B7002C252
:10467A0000300F08E52C452B7002C20F7884E6B48F
:10468A0005057F0412535AE551700875510AD22B59
:06469A0012696B7F05228E
:106D6200200F1590053BE0F54E2024037F0522E518
:0B6D72004ED3940050F3D20F7F0A2292
:105DA5007D077F05124F40500C7D077F05124F4040
:105DB500503230002F7D017F01124F405026D230E6
:105DC5007F01122ECA7F011200167D027F07124F36
:105DD5004050057F04126FF69000A0E0FF7C0A7D1D
:0A5DE500E0125CC51259597F0F222D
:105F510030243DE5484547700C7D087F01124F40D4
:105F610050037F372230030EE53A700A126D987F95
:105F71000112001680173026037F14227884E6B4BC
:105F8100050B7F0312535A2024037F14227F0F2213
:035F91007F142258
:1023400090053DE0F54B7F01126FA2126D987D0262
:102350007F07124F405009E54B70057F04126FE371
:102360009000A1E0FF7C0B7D00125CC5D22B1269AE
:102370006BE545700302246A7C017D001224F25053
:10238000037F3E227C017D501224D250037F3C22E9
:102390007C017D581224D250037F3C227C017D10A9
:1023A0001224DA50081224E250037F33227C017D8C
:1023B000201224DA500B9000BBE0FF7C0E7D4080A1
:1023C000207C017D281224EA500512596F80127C6E
:1023D000017D301224EA50129000B9E0FF7C0E7D9E
:1023E00000125CC512687F7F00227C017D40D229EB
:1023F000E4FF12496A500C7D067F04124F405003DF
:102400007F4C227C017D381224F250037F44227CD1
:10241000017D18C229E4FF12496A500C7D057F0135
:10242000124F4050037F4122E4F55A12594378037A
:10243000C333CE33CED8F912594CE4FF12496A5057
:102440001BAF5A125931C0071259437805C333CE16
:1024500033CED8F9125964D007125C7A055AC3E515
:102460005A648094A840C47F19221224E2500C7D43
:10247000077F05124F40504B3000487884E67004C7
:102480007F0180087884E6B404077F0212535A80E3
:102490002F7884E6B40704760180257D037F061239
:1024A0004F40501CE557455670169000AFE0FF7C3A
:1024B0000C7DC0125CC5900532E0F556A3E0F557DF
:1024C0007F19227D077F05124F4050052000027FB3
:0124D0000506
:1024D10022D229E4FF12496A22D229E4FF12496A71
:1024E100227D077F05124F4022D229E4FF12496A5B
:0924F10022C229E4FF12496A220B
:106C410030260312687F7D077F05124F40500620D2
:0E6C510000037F0522900538E0F54E7F1E22DD
:106B1C00E54E70037F23227D027F07124F40500900
:106B2C00E54B70057F04126FE33024037F0A227F4C
:026B3C001E2217
:106B82001259597D067F01124F40500C9000ACE023
:106B9200FF7C0C7D60125CC5900539E0F54E7F2DBF
:016BA20022D0
:0E6FB0007FA0126FA2900539E0F54E7F2D22D2
:1068F700D22B12696B7D027F07124F405009E54B7F
:1069070070057F04126FE3E54E70037F3222302457
:07691700037F0A227F2D22FD
:10632C00301E037F32227D047F06124F40501FE542
:10633C0055455470199000B0E0FF7C0C7DE0125C68
:10634C00C5900534E0F554A3E0F5557F3222C230F8
:08635C007F01122ECA7F00220E
:106EA10020220CD222E4FF12055BC2227F00227F46
:026EB1003C2281
:106C5F00202218D2227F40120016D201121D87C2A5
:0E6C6F00017F40126FA2C2227F19227F3E22B7
:106F2A0020220A1259791237B3125980227F41223C
:106F3A0020220A1259791261CD125980227F4422E5
:106F4A0020220A1259791255A7125980227F442207
:05000E0000007F052247
:096FFF003025037F0A227F0522E0
:0F6F5A009000A2E0FF7C0B7D20125CC57F0F2210
:0F6F69003025093028037F14227F0F227F142246
:103C51009000A3E0FF7C0B7D40125CC5E54670033C
:103C6100023D297D017F03124F4050707C017D0888
:103C7100C2297F0112496A50037F3F227C017D5096
:103C8100123D2C50037F3D227C017D58123D2C506A
:103C9100037F3D227C017D40D2297F0112496A5078
:103CA1000C7D067F04124F4050037F4D227C017D25
:103CB10028D2297F0112496A500912596F125CC535
:103CC1007F00227C017D18C2297F0112496A500CB4
:103CD1007D057F02124F4050037F43227D027F0307
:103CE100124F405043E4F55AAF5A1259457803C375
:103CF10033CE33CED8F912594C7F0112496A501D87
:103D0100AF5A125931C007AF5A1259457805C3331A
:103D1100CE33CED8F9125964D007125C7A055AC352
:0A3D2100E55A648094A840C07F00BA
:093D2B0022D2297F0112496A220B
:106C7D00202218D222C2307F01122ECA7F01126F3C
:0E6C8D00A27F0112055BC2227F00227F3D2202
:10666E0020222A125987122ECA7FF47E01126D47FC
:10667E007F10120016D202121B86C2027F10126FFA
:10668E00A2C2307F02122ECAC2227F00227F3F2278
:1068CF00202222125987122ECA7FF47E01126D47A1
:1068DF00D2027F011237B3C202C2307F02122ECA18
:0868EF00C2227F00227F432238
:106BA30020221B125987122ECAD2027F011261CDF5
:106BB300C202C2307F02122ECAC2227F00227F4D40
:016BC30022AF
:10561500AF5AEF3395E0FE22900520E0F547A3E071
:10562500F54822900522E0F549A3E0F54A222460D9
:10563500F58274013EAD82FCD2292274702FF58269
:1056450074003EF583E0FF22C202C2227F192224A4
:1056550050F58274053EAD82FC22900536E0F532A8
:10566500A3E0F53322055AC3E55A648094A822D2F3
:0D56750022C2307F0122D222C2307F0222E9
:10326500E5527006126B3E8F5222E552B4050612E6
:1032750036B78F5222E552B40B0612691E8F5222C1
:10328500E552B40A061244788F5222E552B40F066D
:10329500126EB38F5222E552B411061258768F5230
:1032A50022E552B412061251DE8F5222E552B414B1
:1032B50006120A548F5222E552B419061266FD8F82
:1032C5005222E552B41E0612669E8F5222E552B472
:1032D50023061260178F5222E552B42806126FBEDC
:1032E5008F5222E552B42D061262448F5222E552C6
:1032F500B432061263648F5222E552B43C06126E54
:10330500C58F5222E552B43D06126D7D8F5222E5DE
:1033150052B43E06126A008F5222E552B43F06129D
:103325006EE88F5222E552B44106126C048F522288
:10333500E552B44306126AD68F5222E552B44C06C2
:10334500126DB28F5222E552B44D06126AF98F52B0
:1033550022E552B437061257B98F5222E552B439D5
:10336500061255378F5222E552B438061267868FFA
:103375005222E552B43306126B608F5222E552B4E5
:0C3385004406126E148F5222E4F552220E
:106B3E0090052AE0F52BA3E0F52C7D067F02124F7F
:106B4E0040500C90052CE0F529A3E0F52AD21F7FCA
:026B5E0005220E
:1036B700302414201011C21C7D047F01124F40508A
:1036C700037F0B227F0A22302514201211D21C7D82
:1036D700047F02124F4050037F0B227F0A227F088C
:1036E70012640A50061247557F0022202408301022
:1036F70005C2107F0522202508301205C2127F055A
:10370700227D057F06124F40501EE5394538701857
:103717009000B5E0FF7C0D7D80125CC590052EE022
:10372700F538A3E0F53980757D067F06124F4050C6
:103737001EE53C453B70189000B6E0FF7C0D7DA070
:10374700125CC5900530E0F53BA3E0F53C804E7D6B
:10375700077F05124F40500D30000AE52C452B70AE
:1037670004C200800B300F08E52C452B7002C20FF6
:103777007D067F02124F405019301F16E52A452952
:103787007010C21F9000BCE0FF7C0E7D60125CC50C
:10379700800B7884E6B405057F0412535AE551700F
:0C37A7000875510AD22B12696B7F0522B5
:10691E00200F2190053BE0F54E202406201C037F1E
:10692E000522202506301C037F0522E54ED3940058
:07693E0050E7D20F7F0A228F
:104478007D077F05124F4050127D077F05124F4080
:104488004003024529200003024529201C3FD23061
:104498007F03122ECA7F0F126FA290000FE0B402A2
:1044A800047F05800990000FE0B403057F01120026
:1044B8001612561D7D027F07124F4050057F0412C9
:1044C8006FF69000A0E0FF7C0A7DE0804E301C5122
:1044D80090000FE0FF64026005EF640370437F0FF4
:1044E800126FA27F0512640A400BD2307F01122E90
:1044F800CA7F028009D2307F03122ECA7F0A1200B7
:10450800167D027F07124F4050057F04126FF61286
:1045180056289000A2E0FF7C0B7D20125CC57F0F1F
:0A4528002212561D1256287F0F22A2
:106EB300201C063024037F1122301C053025027F5D
:026EC300122299
:10587600302458E5484547700C7D087F01124F409B
:1058860050037F3722300329E53A70257FA0126F37
:10589600A290000FE0B401047F01800990000FE0A0
:1058A600B402057F05120016E4F542C21EC203804B
:1058B600173026037F14227884E6B4050B7F031283
:0E58C600535A2024037F14227F11227F1422C4
:1051DE00301C1030240D20100A7F0A126FA2C21C40
:1051EE007F0A22301C5230254F20124C30030312FE
:1051FE006D98E54A4549700C7D087F02124F40506C
:10520E00037F3822300417E53A70137FA0126FA285
:10521E007F02120016E4F542C21EC2048017302827
:10522E00037F14227884E6B4050B7F0312535A20B1
:10523E0025037F14227F1222201C1230250F2012EC
:10524E000CD21CC2307F02122ECA7F0A227F142279
:100A540090053DE0F54B7F0F126FA2201C0C900017
:100A6400A1E0FF7C0B7D00125CC5301C0C9000A340
:100A7400E0FF7C0B7D40125CC5E542B403037F14A8
:100A840022126D98E4F5427D027F07124F4050090F
:100A9400E54B70057F04126FE3D22B12696B301C97
:100AA40003020B97E5457003020B977C017D00124E
:100AB4000D1E50037F3E227C017D50120CEE50032C
:100AC4007F3C227C017D58120CEE50037F3C227C3B
:100AD400017D10120CF65008120D0650037F3322CC
:100AE4007C017D20120CF65003020BFE7C017D2854
:100AF400120D0E500C9000BAE0FF7C0E7D20020C0B
:100B0400077C017D30120D0E500C9000B9E0FF7C83
:100B14000E7D00020C077C017D40D229E4FF1249BE
:100B24006A500C7D067F04124F4050037F4C227C98
:100B3400017D38120D1E50037F44227C017D18C2B2
:100B440029E4FF12496A500C7D057F01124F405081
:100B5400037F4122E4F55A125615EF7803C333CECE
:100B640033CED8F9125633E4FF12496A501D125697
:100B740015125640C007125615EF7805C333CE330D
:100B8400CED8F9125654D007125C7A12566A40C76E
:100B94007F1922201C03020C8AE5467003020C8A8A
:100BA4007D017F03124F404003020C427C017D080B
:100BB400C2297F0112496A500F7F50120016D230A9
:100BC4007F02122ECA7F3F227C017D50120CFE5000
:100BD400037F3D227C017D58120CFE50037F3D2291
:100BE4007C017D10120D165008120D0650037F3340
:100BF400227C017D20120D1650129000BBE0FF7C78
:100C04000E7D40125CC512687F7F00227C017D400E
:100C1400D2297F0112496A500C7D067F04124F408D
:100C240050037F4D227C017D18C2297F0112496A3D
:100C3400500C7D057F02124F4050037F43227D02FA
:100C44007F03124F40503CE4F55A125615EF7803D7
:100C5400C333CE33CED8F91256337F0112496A50CA
:100C64001D125615125640C007125615EF7805C3CB
:100C740033CE33CED8F9125654D007125C7A1256BA
:100C84006A40C77F1922120D265008120D26504BB8
:100C94003000487884E670047F0180087884E6B4E4
:100CA40004077F0212535A802F7884E6B40704762F
:100CB4000180257D037F06124F40501CE5574556A1
:100CC40070169000AFE0FF7C0C7DC0125CC59005EF
:100CD40032E0F556A3E0F5577F19227D077F051210
:090CE4004F4050052000027F057D
:100CED0022D229E4FF12496A22D229E4FF12496A6D
:100CFD0022D2297F0112496A227D077F05124F40BA
:100D0D0022D229E4FF12496A22D2297F0112496AAF
:100D1D0022C229E4FF12496A227D077F05124F4046
:010D2D0022A3
:1066FD00C219C2307F02122ECA30260512687F8061
:10670D00063028031268A77D077F05124F405006FB
:0F671D002000037F0522900538E0F54E7F1E22F5
:10669E00E54E70037F23227D027F07124F40500983
:1066AE00E54B70057F04126FE33024062010037F44
:1066BE000A22302508201205D21C7F0A227F1E22B4
:10601700201C0512561D80031256287D067F01128B
:106027004F405024E5427020201C0B9000ACE0FF4D
:106037007C0C7D60800C301C0C9000ADE0FF7C0C6C
:106047007D80125CC57F2822900539E0F54E7F2DB3
:016057002226
:0E6FBE007FA0126FA2900539E0F54E7F2D22C4
:10624400D22B12696B7D027F07124F405009E54B38
:1062540070057F04126FE3E54E601D3024062010A4
:10626400037F0A2290000FE06401600930250620B4
:0B62740012037F05227F2D227F3222C3
:10636400301E037F32227D047F06124F40501FE50A
:1063740055455470199000B0E0FF7C0C7DE0125C30
:10638400C5900534E0F554A3E0F5557F3222C230C0
:086394007F01122ECA7F0022D6
:106EC50020220CD222E4FF12055BC2227F00227F22
:026ED5003C225D
:106A000020221FC2307F02122ECAD2227F401200E3
:106A100016D201121D87C2017F40126FA2C2227FCF
:056A200019227F3E2257
:106EE80020220BD222D202121B8612564D227F3F3D
:016EF8002277
:106D7D00202215125674122ECA7F40126FA27F0167
:0B6D8D0012055BC2227F00227F3D2226
:106C040020221912567B122ECA7F10126FA2D201B3
:0F6C1400E4FF1237B3C201C2227F19227F41224F
:106AD60020221D125674122ECA7F40126FA2D23087
:106AE6007F02122ECAD2027F011237B312564D22EE
:036AF6007F4322B9
:106DB20020221412567B122ECAD201E4FF1261CD98
:0A6DC200C201C2227F19227F412284
:106AF90020221D125674122ECA7F40126FA2D23064
:106B09007F02122ECAD2027F011261CD12564D2286
:036B19007F432295
:106E140020221112567B122ECAD202E4FF1255A769
:076E240012564D227F4422AB
:1057B900D2107D027F07124F4050057F04126FE31C
:1057C90090000FE0FF64016004EFB4030E7F011243
:1057D9006FA27F401258087F01801390000FE0B438
:1057E900020F7F05126FA27F501258087F03126FB4
:1057F900E37F50126FA230150312565F7F392212D0
:0F5809000016C22F126A6DE4FD7F0712504F2266
:1055370030241130150BE53345327005C231126A3C
:10554700257F3922E47884F6C21090000FE0FF64CB
:10555700016005EF64037010D2307F01122ECA7FFD
:10556700401255957F01801B90000FE06402701672
:10557700D2307F03122ECA7F05126FA27F501255B9
:10558700957F03122ECA7F50126FA27F002212004E
:1055970016C22F126A6DE4FD7F0812504FC23022E7
:10678600D2127F0A126FA27F40120016D22F126A0F
:106796006DE4FD7F0712504F7F03126FE37F5012A7
:0B67A6006FA230150312565F7F002227
:106B600030000B9000B8E0FF7C0D7DE0800C200031
:106B70000E9000B7E0FF7C0D7DC0125CC5B2007FB7
:026B80001922D8
:1061CD008F5AE55A24FF922F126A6DE55A70127F8D
:1061DD0040120016D201E4FD7F0912504FC201801A
:1061ED0015E55AB401107F10120016D202E4FD7F9E
:0C61FD000912504FC2027F50126FA22204
:10417300C201C202D20C7F50126FA27F80120016BE
:1041830075420390000FE0640170323024297F01EF
:104193001200167D027F07124F4050057F04126FF5
:1041A300F6302404E54270F920240C7F0112422EDC
:1041B30050057F04126FE3E54270D0806490000FD6
:1041C300E0FF64026005EF640370563024357F021C
:1041D300126FA27F051200167F02126FF67D027F17
:1041E30007124F4050057F04126FF6302404E54256
:1041F30070F92024287F0512422E50217F04126F6C
:10420300E3801A3025177F02120016202407302579
:1042130004E54270F62025057F02126FA2E5427085
:10422300AA7FA0126FA2C20CC21E22126FA27D022D
:064233007F07124F40223C
:03000000026CF29D
:106CF200758E0078FEE4F6D8FD9000007FFF7E1FBF
:0D6D0200E4F0A3DFFCDEFA758187024D0985
:10399800C2D530F707B2D563F0FF05F030E70CB2B7
:1039A800D5F4048463F0FF05F080018430D502F477
:0239B8000422E7
:1039BA00EF8DF0A4A8F0CF8CF0A428CE8DF0A42E21
:0239CA00FE22DB
:1039CC00BC000BBE0029EF8DF084FFADF022E4CCDF
:1039DC00F875F008EF2FFFEE33FEEC33FCEE9DECA8
:1039EC00984005FCEE9DFE0FD5F0E9E4CEFD22EDEE
:1039FC00F8F5F0EE8420D21CFEADF075F008EF2F38
:103A0C00FFED33FD4007985006D5F0F222C398FD28
:053A1C000FD5F0EA22C5
:103A2100EB9FF5F0EA9E42F0E99D42F0E89C45F0FB
:013A31002272
:103A32007401FF3395E0FEFDFC080808E6CF2FF67F
:103A420018E6CE3EF618E6CD3DF618E6CC3CF62258
:0C3A5200A42582F582E5F03583F583227F
:103A5E00D083D082F8E4937012740193700DA3A3F7
:103A6E0093F8740193F5828883E47374029368600B
:063A7E00EFA3A3A380DF0B
:106EF900EFC39461400AEF947B5005EF24E0FF2231
:016F09002265
:00000001FF
